:020000040000FA
:040200006BEF03F0AD
:040208000EEF01F004
:080218002DEF01F0D8CF01F039
:10022000E0CF02F0006EF3CF03F0F4CF04F0F0ACB7
:100230001DEF01F0F0B066EC0BF0A2A023EF01F08F
:10024000A1B018EC09F003C0F3FF04C0F4FF0050A4
:1002500002C0E0FF01C0D8FF1000D8CF06F0E8CF01
:1002600005F0E0CF07F0F3CF08F0F4CF09F0F0BCD1
:100270003DEF01F0F0B066EC0BF0A2B043EF01F0FF
:10028000A1B018EC09F0A2B04CEF01F0AECFE8FF3E
:100290006ECFE8FF52EF01F09EBA0CEC0FF0A4BA5B
:1002A00077EC0FF008C0F3FF09C0F4FF07C0E0FFD0
:0A02B00005C0E8FF06C0D8FF1000EB
:10030000F95000011150F926CEEF29F0D0EF29F075
:10031000DDEF29F0F2EF29F000EF2AF00EEF2AF0DE
:100320001CEF2AF02AEF2AF03AEF2AF048EF2AF0E1
:1003300056EF2AF012000009D8A4A5EF01F0000141
:10034000000E0F6E000E106E1200E806030B0A0D71
:10035000F9CFE8FFF350F92683C00FF084C010F006
:10036000120085C00FF086C010F0120087C00FF099
:1003700088C010F0120089C00FF08AC010F012007F
:10040000EFCFE8FFE806070B0A0DF9CFE8FFF3503E
:10041000F9263CC04EF03DC04FF012003AC04EF0FD
:100420003BC04FF012003EC04EF03FC04FF01200F4
:1004300040C04EF041C04FF0120042C04EF043C0E9
:100440004FF0120044C04EF045C04FF0120046C0BD
:100450004EF047C04FF0120048C04EF049C04FF078
:1004600012000F0B060DF9CFE8FFF350F926BBC2BF
:10047000E8FF1200BCC2E8FF1200BDC2E8FF120094
:10048000BEC2E8FF1200BFC2E8FF1200C0C2E8FF10
:100490001200C1C2E8FF1200C2C2E8FF1200C3C2CC
:1004A000E8FF1200C4C2E8FF1200C5C2E8FF120054
:1004B000C6C2E8FF1200C7C2E8FF1200C8C2E8FFC8
:0E04C0001200C9C2E8FF1200CAC2E8FF120013
:100500000001E806070B0A0DF9CFE8FFF350F926C2
:100510008D510D6E8E510E6E12008F510D6E9051D9
:100520000E6E120091510D6E92510E6E120093518B
:100530000D6E94510E6E120095510D6E96510E6E09
:10054000120097510D6E98510E6E120099510D6E5A
:100550009A510E6E12009B510D6E9C510E6E120040
:100600000001E8BE33EF03F0E806070B0A0DF9CF4F
:10061000E8FFF350F9260D5073270E507423120093
:100620000D5075270E50762312000D5077270E506F
:10063000782312000D5079270E507A2312000D50A6
:100640007B270E507C2312000D507D270E507E23F9
:1006500012000D507F270E50802312000D5081276D
:100660000E5082231200E806070B0A0DF9CFE8FFAF
:10067000F350F9260D50736F0E50746F12000D5029
:10068000756F0E50766F12000D50776F0E50786FA9
:1006900012000D50796F0E507A6F12000D507B6F63
:1006A0000E507C6F12000D507D6F0E507E6F120049
:1006B0000D507F6F0E50806F12000D50816F0E50E5
:1006C000826F1200F2AE12000001010EA16FA1674D
:1006D00067EF03F0120092988098939C819C000130
:1006E0005B6A5C6A640E9DEC0BF092988098000146
:1006F000546A640E9DEC0BF00F018350306E316E26
:10070000326E0F018450336E346E356E0F01999046
:10071000878094969394829681940001000E176EC0
:10072000000E186E0001000E196E000E1A6E000108
:10073000000E1B6E000E1C6E0001000E1D6E000EE2
:100740001E6E0001000E136E000E146E0001000EEE
:10075000156E000E166E0001000EAB6F000EAC6F32
:100760000001000EAD6F000EAE6F0001000EAF6F06
:10077000000EB06F0001000EB16F000EB26F0001ED
:100780005E6A5F6A606BA16BA26BA36BE769E96B42
:100790000201BA6B0101116B0001CC6B91EC31F0DD
:1007A000020100510001A56F040E93EC08F0040E45
:1007B00093EC08F00001C350C56FC450C66F050E1E
:1007C00093EC08F0050E93EC08F00001C350C76FDE
:1007D000C450C86F000EE8CF0DF0E86AE8CF0EF005
:1007E000A8EC0BF0E8CF00F5010EE8CF0DF0E86AB9
:1007F000E8CF0EF0A8EC0BF0E8CF01F5C0EC0CF060
:10080000FA0E9DEC0BF0FA0E9DEC0BF0FA0E9DEC3F
:100810000BF0FA0E9DEC0BF0C8EC08F0C7EC24F0DE
:10082000A5EC0EF0B9EC0EF0F28EF28CD08E0F012A
:10083000D89083B6D880D8B023EF04F00A0E9DEC90
:100840000BF00F01D89083B6D880D8B039EF04F000
:100850000F01D89084B2D880D8B034EF04F00A0EDB
:100860009DEC0BF00F01D89084B2D880D8A05BEF3C
:1008700004F094EC1EF00201A50EA76346EF04F00D
:10088000E70EA86346EF04F04AEF04F091EC31F074
:10089000C9EC0BF000C2E8FF0FEC1FF00301AD51F3
:1008A0000201A56FE9EC0AF064EC0AF00101F20E16
:1008B000066FA1EC0AF00F01D89084B2D880D8A0BE
:1008C0005BEF04F00A0E9DEC0BF00F01D89084B2A0
:1008D000D880D8A05BEF04F00F01D89084B4D88002
:1008E000D8B078EF04F00A0E9DEC0BF00F01D89011
:1008F00084B4D880D8B08EEF04F00F01D89083B6BE
:10090000D880D8B089EF04F00A0E9DEC0BF00F01EF
:10091000D89083B6D880D8A0BBEF07F00201A0C260
:100920000AF00201FF0E0AB0A56FA561FBEF04F00B
:100930000301A6A1DBEF04F00F0183BEDBEF04F09F
:10094000800E0FEC0DF0000EF86E640EF76E920E36
:10095000F66E85EC0DF0C00E0FEC0DF0000EF86E8B
:10096000640EF76E380EF66E85EC0DF00F01D89020
:1009700084B4D880D8B0C2EF04F00A0E9DEC0BF01E
:100980000F01D89084B4D880D8B0B6EF04F00F012E
:10099000D89084B4D880D8A0C7EF04F00A0E9DEC9C
:1009A0000BF00F01D89084B4D880D8A0C7EF04F022
:1009B000C80E9DEC0BF00201D1B1E2EF04F0D1A31F
:1009C000FBEF04F0800E00019D6FA8EC30F0D89092
:1009D0002EEC27F0D8B0F2EF04F00201FF0EA56F65
:1009E000FBEF04F0E9EC0AF064EC0AF0A1EC0AF089
:1009F0000A0E9DEC0BF00001010E366EA3C252F000
:100A0000A4C253F00201A25100014D6E6AEC23F022
:100A100067EC1FF0FCAE10EF05F00F01939481948A
:100A2000000133B030EF05F0010E366296EF05F0AD
:100A30000001050EE8CF5DF0070E37EC0AF0020E5C
:100A4000366E0001A5510201006329EF05F096EF13
:100A500005F0006F0FEC1FF067EC1FF096EF05F04C
:100A6000010E366E0BEC23F0FDEC17F040EC07F0B6
:100A70000201A1A161EF05F00301B6517FEC24F062
:100A8000D8A061EF05F00201B76759EF05F0ABC0E0
:100A900073F0ACC074F0ADC075F0AEC076F0AFC00E
:100AA00077F0B0C078F0B1C079F0B2C07AF061EF01
:100AB00005F0F08CF086A290E868E8CFEEF067EFE2
:100AC00005F0F09CF086A280E86AE8CFEEF0020123
:100AD000A0B186EF05F02FEC17F0D8B486EF05F043
:100AE000B3EC19F046EC19F080EC1BF012EC1CF0A2
:100AF00011EC1AF0A0EC21F0BFEC1FF0A8EC21F0F3
:100B0000F7EC1AF00001E9673CEC10F062EC03F03E
:100B1000F3EC1CF05EEC0EF00001A26794EF05F020
:100B20000A0EA26FDEEC05F00AEF05F0800E0FEC66
:100B30000DF0000EF86E650EF76EC40EF66E85ECC5
:100B40000DF0C00E0FEC0DF0000EF86E640EF76E97
:100B5000380EF66E85EC0DF083EC1EF0D8A0B3EFE6
:100B600005F041EC25F0FDEC17F0B3EC19F046EC84
:100B700019F080EC1BF012EC1CF011EC1AF0A0EC58
:100B800021F0BFEC1FF0A8EC21F0F7EC1AF0F3EC29
:100B90001CF05EEC0EF00AEF05F00001100E0B6E7B
:100BA000C00E0FEC0DF0000EE16E030EE26EE6508B
:100BB00000EC0DF00B2ED7EF05F012000001840EB3
:100BC0000FEC0DF0200E00EC0DF00201520EA5BF4F
:100BD000200E000100EC0DF00601CE517FEC24F058
:100BE000410ED8A0200E00EC0DF00301B2517FECB5
:100BF00024F04D0ED8B02D0E00EC0DF00301B351D2
:100C00007FEC24F04D0ED8B02D0E00EC0DF003015A
:100C1000B4517FEC24F04D0ED8B02D0E00EC0DF049
:100C2000200E00EC0DF0800E0FEC0DF0B9C20DF0AF
:100C3000BAC20EF00E6A0001640E0F6E000E106E46
:100C400067EC10F013C011F014C012F08BC00DF05F
:100C50008CC00EF013C20FF014C210F067EC10F04D
:100C60001450E8CF13F01550E8CF14F0156A0101C5
:100C700011B14BEF06F000011150135C12501458E3
:100C8000E8AE4BEF06F0C90E00015D6E050E37ECC5
:100C90000AF001011169000115EC0EF0200EE8CFF9
:100CA0000AF0300E25640AC025F0255000EC0DF046
:100CB000265000EC0DF02E0E00EC0DF0275000EC4D
:100CC0000DF00301B6517FEC24F0D8A071EF06F0CF
:100CD000800E0FEC0DF000C513F001C514F0EBEC25
:100CE0000DF00201B8AF8AEF06F0B86B000EE8CF46
:100CF0000DF0E86AE8CF0EF000C5E8FFB3EC0BF0AA
:100D0000010EE8CF0DF0E86AE8CF0EF001C5E8FF6C
:100D1000B3EC0BF069EC07F0D8B0B4EF06F07AEC66
:100D200007F0D8B0B4EF06F0CCEC24F0D8B0B4EFB4
:100D300006F09EEC23F00001A351E812D8A4B4EF12
:100D400006F00201A0A1B2EF06F0C00E0FEC0DF00C
:100D5000000EF86E640EF76E520EF66E85EC0DF016
:100D6000B4EF06F0CDEC05F0000133B4CFEF06F0A0
:100D700035A4CFEF06F03594010E5D6E050E37EC0D
:100D80000AF000015466CEEF06F0542ABEC358F0B4
:100D9000BFC359F0CA6BCB6BCFEF06F0540600010E
:100DA00054A002EF07F0596602EF07F03B0E5A62BB
:100DB000E1EF06F0050E5D6E0A0E37EC0AF002EF69
:100DC00007F01E0E5A62ECEF06F0030E5D6E0A0E7F
:100DD00037EC0AF002EF07F00A0E5A62F7EF06F05E
:100DE000010E5D6E0A0E37EC0AF002EF07F0060EF8
:100DF0005A6002EF07F0010E5D6E0A0E37EC0AF042
:100E000002EF07F07F0E5A6E5650CE6F5750CF6FDD
:100E1000010E54622BEF07F058505910D8B41AEF56
:100E200007F05850CE6F5950CF6F000E0301BD63CD
:100E30002BEF07F0020E0301BD5DD8B427EF07F0DA
:100E40000001CA51CE6FCB51CF6F2BEF07F0E86A8C
:100E50000001CE6FCF6F00018B0E0FEC0DF0CF5164
:100E6000E8CF13F0146A156A166AE3EC0DF03A0E37
:100E700000EC0DF0CE51E8CF13F0E3EC0DF01200D2
:100E80000301C0517FEC24F0D8A066EF07F0030106
:100E9000000EC16563EF07F000017ABF66EF07F04F
:100EA0000301C15100010D6E0E6A00010A0E0F6EA2
:100EB000000E106E67EC10F07951135E7A51145CDD
:100EC000D8B066EF07F00001E76912000001E76B98
:100ED0001200D8900001CCAF1200C00E0FEC0DF044
:100EE000000EF86E640EF76EFE0EF66E85EC0DF0D9
:100EF000D88012000D0E93EC08F00D0E93EC08F064
:100F000069C00DF06AC00EF0A9C20FF0AAC210F0BD
:100F100067EC10F000011450136E1550146E16504B
:100F2000156E166A15EC0EF00001255026100F0BF9
:100F3000D890D8B41200C00E0FEC0DF0000EF86E71
:100F4000640EF76EEC0EF66E85EC0DF0CB0E0FEC2A
:100F50000DF00001255000EC0DF0265000EC0DF0D6
:100F60002E0E00EC0DF0275000EC0DF0285000EC98
:100F70000DF0D88012000F01D89084B4D880D8A08A
:100F8000BBEF07F00A0E9DEC0BF00F01D89084B474
:100F9000D880D8A0BBEF07F00F01D89083B6D880D7
:100FA000D8A0CCEF07F00A0E9DEC0BF00F01D89003
:100FB00083B6D880D8A0CCEF07F0800E0FEC0DF0F0
:100FC0000F018350A2EC0DF00F018450A2EC0DF044
:100FD000C00E0FEC0DF00F018650A2EC0DF00F01CA
:100FE0008750A2EC0DF00F01835082868184E8B017
:100FF0008296E8B281948098E8B48088320E9DECA5
:101000000BF00F01D89084B4D880D8B00DEF08F061
:101010000A0E9DEC0BF00F01D89084B4D880D8B0A4
:10102000DDEF07F00F01D89084B4D880D8A012EF7C
:1010300008F00A0E9DEC0BF00F01D89084B4D88014
:10104000D8A012EF08F0C00E0FEC0DF0000EF86EF5
:10105000630EF76EA80EF66E85EC0DF000010D6ABA
:10106000800E0FEC0DF0000EF86E630EF76EDE0EC4
:10107000F66E85EC0DF0870E0FEC0DF000010D50B3
:10108000AFEC0DF093EC08F08C0E0FEC0DF00F01AF
:10109000C4CFE8FFAFEC0DF00F01C3CFE8FFAFEC1A
:1010A0000DF0320E9DEC0BF00F01D89084B4D88077
:1010B000D8B060EF08F00A0E9DEC0BF00F01D8904D
:1010C00084B4D880D8B030EF08F00F01D89084B441
:1010D000D880D8A065EF08F00A0E9DEC0BF00F0148
:1010E000D89084B4D880D8A065EF08F000010D2A0C
:1010F0000C0E0D6430EF08F0DDEF07F00001136A0D
:10110000146A156A166A0A6E0B6A0A5093EC08F0A4
:101110000001C3501326C4501422D8B0152A0B2E38
:1011200085EF08F012000A6EA10EC06E000EC16EAF
:101130000AC0E8FF31EC02F0E8AEC188E89EE8445E
:10114000E844C26EC2800000C282C2B2A5EF08F0BD
:101150000001C3CF69F0C4CF6AF00AC0E8FF1200F3
:101160000F01C282C2B2B2EF08F00001C35069277A
:10117000C4506A23120093EC08F0B0EC08F0B0EC15
:1011800008F0B0EC08F000016A336A9F693312007E
:1011900000014C6A566A576A280EE8CF55F00001E4
:1011A000900E526E010E536E0001900E4E6E010EA7
:1011B0004F6E506A516A100E0001E8CF4DF0386A48
:1011C0003A6A3C6A3E6A406A426A446A466A486AC7
:1011D0004A6A080EE8CF39F0E8CF3BF0E8CF3DF09F
:1011E000E8CF3FF0E8CF41F0E8CF43F0E8CF45F05B
:1011F000E8CF47F0E8CF49F0E8CF4BF0979E858ED7
:10120000000152500F01E8CFBBFF010153500F0105
:10121000E8CFBCFF0A0E0F01E8CFBAFF0F01A08094
:101220000F019E900F01080EE8CFB1FFB1801200B0
:101230000001EEA1857E0201BAAF22EF09F08770AE
:101240002AEF09F00001E5B129EF09F087802AEFC4
:1012500009F087900001BBCFE8FF4E26BCCFE8FF26
:101260004F224EC0E8FFE8CFBBFF4FC0E8FFE8CFFA
:10127000BCFF0001E86A4C64A1EC09F000014C2AB3
:101280004CC0E8FFFE0B4D6057EF09F04C6A500E62
:10129000E8CF4EF050C0E8FF4E5EC30EE8CF4FF0EF
:1012A00051C0E8FF4F5A506A516A9EEF09F04CA0B6
:1012B0006CEF09F052C0E8FFE8CF4EF053C0E8FFF2
:1012C000E8CF4FF0BAC2E8FF0001E5814C6298EF29
:1012D00009F0E59198EF09F0120E4C6284EF09F0E5
:1012E00050C0E8FFE8CF4EF051C0E8FFE8CF4FF024
:1012F0004F324E324F324E324F324E324F324E32EA
:101300000F0E4F1698EF09F0040EE8CFEAFF000E1B
:10131000E8CFE9FF4CC0E8FFE830E89EE804E926A2
:1013200000EC02F052C0E8FF4E5E53C0E8FF4F5A97
:101330004EC0E8FF50264FC0E8FF51220F01A19098
:10134000120093EC0EF09DEC0EF00001010E3662DF
:10135000B0EF09F000018286BDB18296FF0EBD6F2D
:1013600087900301CDBFB8EF09F0859EB9EF09F072
:10137000858E0001552EFFEF09F0CAEC24F0000124
:1013800054A0EFEF09F00001FF0EE763EFEF09F063
:1013900058C0E8FF5910D8B4E7EF09F05866D4EF09
:1013A00009F03C0E586E5906580658505A6E030103
:1013B000E86ABD11D8B4E7EF09F0000158505910A0
:1013C000D8B4E7EF09F0CA6BCB6BEFEF09F000017F
:1013D000CA2B3C0ECA63EFEF09F0CA6BCB2B280E69
:1013E000E8CF55F0562A3C0E5662FFEF09F0566AD8
:1013F000572A0501002BD8B4012B0201B86902015C
:10140000A1A108EF0AF0530EC5EC0EF00001A86B85
:10141000000183CFE8FF311AD8A4306E316E30C09E
:10142000E8FF3212000184CFE8FF341AD8A4336EEB
:10143000346E33C0E8FF351200015E665E065F66FB
:101440005F0660676007A167A107A267A207A3679D
:10145000A3075C662DEF0AF012005C2E1200807864
:101460005D4E12005BC0E8FFE8CF5CF01200E8CFF1
:101470005BF0E8CF5CF08088120000010ABE44EF08
:101480000AF0819E45EF0AF0818E828A829A0A468E
:101490000B2E3DEF0AF012000201AD510A6E080E4C
:1014A0000B6E3DEC0AF00201AC510A6E080E0B6E99
:1014B0003DEC0AF00201AB510A6E080E0B6E3DECDA
:1014C0000AF08686869612000BC113F00CC114F048
:1014D0000DC115F009C117F00AC118F06BEC11F03D
:1014E0000201A55101010F03F35000011326D8B0EA
:1014F000142AD8B0152A0101006B016B026B0001A0
:101500001350E846E846E880E8921F0B13B6E88ED1
:101510000101006F000113361436153613361436E8
:101520001536133614361536133614361536145050
:101530000101016F000115501F0B01011009026F1D
:10154000120064EC0AF0010108510A6E080E0B6EDD
:101550003DEC0AF0010107510A6E080E0B6E3DECDE
:101560000AF0010106510A6E080E0B6E3DEC0AF0FE
:1015700086868696010105510A6E080E0B6E3DECBB
:101580000AF0010104510A6E080E0B6E3DEC0AF0E0
:10159000010103510A6E080E0B6E3DEC0AF08686BF
:1015A0008696010102510A6E080E0B6E3DEC0AF0A0
:1015B000010101510A6E080E0B6E3DEC0AF00101AB
:1015C00000510A6E080E0B6E3DEC0AF08686869678
:1015D00012000F01939E949A939C819C819E829A03
:1015E000989686960201D1A118EF0BF0D1B318EFAF
:1015F0000BF004C206F105C207F106C208F101C2F0
:1016000003F102C204F103C205F10101700E0B6F78
:10161000C60E0C6F000E0D6F0101140E096F000E47
:101620000A6F01010E6B0A0E106F010E0F6F120090
:101630000201D1B13EEF0BF0D1A33EEF0BF00AC295
:1016400006F10BC207F10CC208F107C203F108C290
:1016500004F109C205F101016C0E0B6FCF0E0C6F86
:10166000000E0D6F0101640E096F000E0A6F01017B
:101670000E6B080E106F010E0F6F12000201D1B138
:1016800065EF0BF0D1B365EF0BF010C206F111C29C
:1016900007F112C208F10DC203F10EC204F10FC22C
:1016A00005F101014A0E0B6F190E0C6F010E0D6F43
:1016B00001010A0E096F000E0A6F01010B0E0E6F79
:1016C000320E106F020E0F6F1200120087B284EFFD
:1016D0000BF0D5AE76EF0BF0D6CFC1F0D7CFC2F07E
:1016E0000001C32BD8B4C42BF09012000001C351E9
:1016F000C411F090D8A41200E86AE8CFD7FFE8CF71
:10170000D6FFD58EF0901200F17AF0AC96EF0BF088
:101710000301CDA192EF0BF0F1AA859EF1BA858E5F
:1017200096EF0BF0F1AA858EF1BA859EF09012002B
:101730000000E82E98EF0BF012000A6EFA0E98ECFB
:101740000BF0FA0E98EC0BF00A2E9EEF0BF0120045
:101750000EC0E8FFAA6E0DC0E8FFA96EA69EA69C6B
:10176000A680A8501200A86E0EC0E8FFAA6E0DC099
:10177000E8FFA96EA69EA69CA684F29E550EA76EB3
:10178000AA0EA76EA682F28EA1A8C4EF0BF0A198B4
:101790001200800E0FEC0DF0000EF86E640EF76E66
:1017A000A40EF66E85EC0DF0C00E0FEC0DF0000EE1
:1017B000F86E640EF76E260EF66E85EC0DF077EC83
:1017C00027F0D8A009EF0CF0C00E0FEC0DF0000EC2
:1017D000F86E640EF76EB60EF66E85EC0DF091ECB9
:1017E00031F0A9EC1EF00001600E9E6F00C2E8FF10
:1017F0003AEC1FF00201002B0301072B3A0E07639E
:1018000005EF0CF0062B300E076F00019E2FF6EF50
:101810000BF094EC1EF000C2E8FF0FEC1FF012007A
:1018200000011550F86E1450F76E1350F66E00015B
:101830000E50E26E0D50E16E0900F550E66E0A069C
:101840000900F550E66E0A2E1CEF0CF012000001A4
:101850001550F86E1450F76E1350F66EA68EA69CB7
:10186000A684A688F29E550EA76EAA0EA76EA68223
:101870000000F28E0001400E1326000E14221522E5
:101880000A2E27EF0CF0120062EC03F00001155055
:10189000F86E1450F76E1350F66EA68EA69CA684B2
:1018A000A688F29E550EA76EAA0EA76EA682F28E8D
:1018B0000A0000010E50E26E0D50E16E400E0B6EFC
:1018C000E6CFE8FFF56E0F000B2EFAD7A68EA69C8A
:1018D000A684F29E550EA76EAA0EA76EA682F28E61
:1018E000A6940001400E1326000E142215220001BA
:1018F000400E0D26000E0E220A2E44EF0CF01200B0
:1019000000011550F86E1450F76E1350F66EA68E47
:10191000A69CA684A688F29E550EA76EAA0EA76E58
:10192000A6820000F28E0A00080E0B6E00010E5017
:10193000E26E0D50E16E080E0C6EE6CFE8FFF56E1C
:101940000F000C2EFAD7A68EA69CA684F29E550EEA
:10195000A76EAA0EA76EA6820000F28E0B2EEBD702
:10196000A6940001400E1326000E14221522000139
:10197000400E0D26000E0E220A2E80EF0CF01200F3
:101980000F019A6A886A9396939A93988186818ABE
:101990008188140E9DEC0BF0380E0FEC0DF0050E47
:1019A0009DEC0BF0380E0FEC0DF0010E9DEC0BF0E2
:1019B000380E0FEC0DF0010E9DEC0BF0380E0FEC15
:1019C0000DF0060E0FEC0DF00E0E0FEC0DF0010EEB
:1019D0000FEC0DF0800E0FEC0DF0800E0FEC0DF003
:1019E000630EF76EBA0EF66E85EC0DF0C00E0FECBE
:1019F0000DF0630EF76ECC0EF66E85EC0DF0120056
:101A00001EEC0DF032EC0DF0818A81980000000090
:101A100081860000000081960000000012001EEC8C
:101A20000DF032EC0DF0819A819800000000818663
:101A300000000000819600000000120025EC0DF06F
:101A4000D8B01EEF0DF09A6A12009A688188819AC8
:101A500000000000818600000000D89088B0D88087
:101A600081961200886AE8B08888E8B2888AE8B46B
:101A7000888CE8B6888EE8B88886E8BA8884E8BC9E
:101A80008882E8BE8880120010101010101010100C
:101A900018181818181818181C1C1C1C1C1C1C1CA6
:101AA0001E1E1E1E1E1E1E1E01010101010101013E
:101AB00003030303030303030707070707070707D6
:101AC0000F0F0F0F0F0F0F0F800E0FEC0DF00DC04B
:101AD000F6FF0EC0F7FFF86A85EC0DF01200C00E9D
:101AE0000FEC0DF00DC0F6FF0EC0F7FFF86A85ECA5
:101AF0000DF01200C00E0FEC0DF0CEC0F6FFCFC0FF
:101B0000F7FFF86A85EC0DF01200100E88EF0DF06B
:101B10000A6E0900F5CFE8FFE812D8B4A1EF0DF086
:101B200000EC0DF00A4EA1EF0DF00900F5CFE8FF33
:101B3000E812D8B4A1EF0DF000EC0DF00A2E89EFF9
:101B40000DF012000A6E080E0B6E300E0ABE310E3A
:101B500000EC0DF00A360B2EA5EF0DF012000A6E08
:101B60003A0E0B6E0AC0E8FFF00BE842E842E8428A
:101B7000E84230090B64070F00EC0DF00AC0E8FFE3
:101B80000F0B30090B64070F00EC0DF00AC0E8FFE3
:101B9000120015EC0EF0255000EC0DF0265000EC74
:101BA0000DF0275000EC0DF0285000EC0DF02950FE
:101BB00000EC0DF0120015EC0EF0CEEF0DF015EC70
:101BC0000EF0D1EF0DF015EC0EF0D4EF0DF015EC9A
:101BD0000EF0D7EF0DF015EC0EF0FFEC0DF02550E8
:101BE00000EC0DF0265000EC0DF0275000EC0DF04D
:101BF000285000EC0DF0295000EC0DF0120000010F
:101C0000300E25621200200E256E300E2662120064
:101C1000200E266E300E27621200200E276E300E28
:101C200028621200200E286E12000001196A1A6A3A
:101C3000100E176E270E186E6BEC11F0300E13108D
:101C4000256E1BC013F01CC014F01DC015F01EC083
:101C500016F0196A1A6AE80E176E030E186E6BEC0E
:101C600011F0300E1310266E1BC013F01CC014F0C0
:101C70001DC015F01EC016F0196A1A6A640E176EA0
:101C8000000E186E6BEC11F0300E1310276E1BC097
:101C900013F01CC014F01DC015F01EC016F0196A18
:101CA0001A6A0A0E176E000E186E6BEC11F0300EE9
:101CB0001310286E300E1B10296E12000001310E19
:101CC000376267EF0EF094EC1EF091EF0EF0320EDB
:101CD000376271EF0EF000C2E8FF0FEC1FF091EFDA
:101CE0000EF0330E376279EF0EF0A9EC1EF091EF93
:101CF0000EF0340E376281EF0EF000C2E8FF3AECCE
:101D00001FF0350E376291EF0EF00001FF0E0D6EE1
:101D1000030E0E6EE8CF0EF0FF0EB3EC0BF091EF5A
:101D20000EF0376A12000F01ABA21200AB98AB881D
:101D30000F01AE500001616B12000F016BA2120087
:101D40006B986B880F016E5012000C0EE8CFAFFF3E
:101D5000220EE8CFACFF900EE8CFABFF0001616B25
:101D60009F9A9D8A1200ACA2B3EF0EF0E8CFADFFB0
:101D70001200000EE8CF6FFF220EE8CF6CFF900E2E
:101D8000E8CF6BFFA59AA38A12006CA2C5EF0EF0F4
:101D9000E8CF6DFF1200E1CF21F0E2CF22F0000189
:101DA00065C0E1FF000164C0E2FF686BACA2D6EF42
:101DB0000EF0E6CFE8FF00016827E8CFADFF000195
:101DC000662FD6EF0EF021C0E1FF22C0E2FF120025
:101DD000E1CF21F0E2CF22F0000165C0E1FF000178
:101DE00064C0E2FF686B0001050E5E6EE86A5E6427
:101DF00007EF0FF09EAAF7EF0EF0AECFE8FFE8CFA7
:101E0000E6FF000168270001662FF3EF0EF021C006
:101E1000E1FF22C0E2FF12009EAA12000001000EA4
:101E200061631FEF0FF0AECFE8FFE8CF62F0550E11
:101E300062631200280EE8CF5FF0612B1200010EE2
:101E4000616329EF0FF0AECFE8FFE8CF63F0612BBD
:101E50001200020E616333EF0FF0AECFE8FFE8CF60
:101E600064F0612B1200030E61633DEF0FF0AECF03
:101E7000E8FFE8CF65F0612B1200040E616346EFC6
:101E80000FF0AECFE8FFE8CF66F0612B050E61637F
:101E900052EF0FF0010E636350EF0FF0E8EC0EF01D
:101EA000612B1200060E616375EF0FF0AECFE8FFF5
:101EB000E8CF67F0020E636366EF0FF0CBEC0EF035
:101EC00068C0E8FFB3EC0EF0616B120068C0E8FF79
:101ED000676370EF0FF00C0EB3EC0EF0616B120045
:101EE0000D0EB3EC0EF0616B1200616B1200A4AA30
:101EF00012006ECFE8FF0201A1B1ABEF0FF0530A61
:101F0000D8A412000201A0A1120000010F0E741546
:101F10001009C5EC0EF073C0E8FFC5EC0EF000012F
:101F20000F0E76152009C5EC0EF07551C5EC0EF0BC
:101F300000010F0E78153009C5EC0EF07751C5EC95
:101F40000EF000010F0E7A154009C5EC0EF0795124
:101F5000C5EC0EF012000001A8B1B2EF0FF0AA6FAD
:101F6000A82B1200A96FA82B020EA863CBEF0FF0CD
:101F7000AA51F00B100AD8A410EF10F00F0EAA17F8
:101F8000AAA7C5EF0FF0F00EAA13A9C0ABF0AAC024
:101F9000ACF010EF10F0040EA863E2EF0FF0AA51BE
:101FA000F00B200AD8A410EF10F00F0EAA17AAA762
:101FB000DCEF0FF0F00EAA13A9C0ADF0AAC0AEF08E
:101FC00010EF10F0060EA863F9EF0FF0AA51F00B16
:101FD000300AD8A410EF10F00F0EAA17AAA7F3EF3B
:101FE0000FF0F00EAA13A9C0AFF0AAC0B0F010EF26
:101FF00010F0080EA86310EF10F0AA51F00B400A81
:10200000D8A410EF10F00F0EAA17AAA70AEF10F02D
:10201000F00EAA13A9C0B1F0AAC0B2F010EF10F0F0
:1020200012000C0E0F016F6E220E6C6E900EE8CF38
:102030006BFF12000001E80E0D26030E0E22780E33
:102040000D5C070E0E58D8A029EF10F0EF0E30EF00
:1020500010F00E320D320E320D320E320D320D50A6
:10206000C5EF0EF0BC0E0D5C030E0E58D8A02BEF82
:1020700010F0EF0E30EF10F0F00EC5EC0EF0800E09
:10208000C5EC0EF073C00DF074C00EF01AEC10F039
:1020900075C00DF076C00EF01AEC10F077C00DF0A0
:1020A00078C00EF01AEC10F079C00DF07AC00EF086
:1020B00032EC10F07BC00DF07CC00EF032EC10F072
:1020C0007DC00DF07EC00EF032EC10F0120078EC06
:1020D00010F010AE70EF10F00D50155E0E50165A45
:1020E0000EAE77EF10F00F50155E1050165A12001A
:1020F0000001136A146A156A166A0F500D02F3CFB5
:1021000013F0F4CF14F00F500E02F3501426F450D5
:102110001522D8B0162A10500D02F3501426F45090
:102120001522D8B0162A10500E02F3501526F4507E
:10213000162212000001246A1B6A14501310D8B42E
:10214000000C14501718E8BE241EA46B000E17AE26
:10215000ACEF10F0171E172A14AEB3EF10F0131ED9
:10216000141E132A142214501710E8BE3FEF11F06A
:1021700017501B5E143614341B3617501B261436AA
:1021800014341B36175014B01B5E14A01B261436D3
:1021900014341B36175014B01B5E14A01B261436C3
:1021A00014341B36175014B01B5E14A01B261436B3
:1021B00014341B36175014B01B5E14A01B261436A3
:1021C00014341B36175014B01B5E14A01B26143693
:1021D00014341B36175014B01B5E14A01B26143683
:1021E00013341B36175014B01B5E14A01B26133675
:1021F00013341B36175013B01B5E13A01B26133667
:1022000013341B36175013B01B5E13A01B26133656
:1022100013341B36175013B01B5E13A01B26133646
:1022200013341B36175013B01B5E13A01B26133636
:1022300013341B36175013B01B5E13A01B26133626
:1022400013341B36175013B01B5E13A01B26133616
:1022500013341B36175013B01B5E13A01B26133606
:1022600013A01B26A4B15DEF11F024AE000C131EC9
:10227000141EE86A132A14221B1E1B2A000C17AE18
:1022800058EF11F014BE54EF11F0E8CF9DF0135049
:10229000E8CF1BF01B9E133614361450E8CF13F012
:1022A0009D51146A35EF11F0136A132A146A000C59
:1022B000141E131EA42BB8EF10F01B2A17501B621C
:1022C00035EF11F01B6A000E132A142214AE35EFFD
:1022D00011F02388FF0C0001246A1C6A1B6A155048
:1022E00014101310D8B4000C15501818E8BE241E92
:1022F000A46B000E18AE81EF11F0171E181E172ADE
:10230000182215AE8AEF11F0131E141E151E132A83
:102310001422152215501810E8BE14EF13F01750B0
:102320001B5E18501C5A153615341B361C361750B8
:102330001B2618501C22153615341B361C36175018
:1023400015A0A8EF11F01B5E18501C5AABEF11F04E
:102350001B2618501C22153615341B361C361750F8
:1023600015A0B8EF11F01B5E18501C5ABBEF11F00E
:102370001B2618501C22153615341B361C361750D8
:1023800015A0C8EF11F01B5E18501C5ACBEF11F0CE
:102390001B2618501C22153615341B361C361750B8
:1023A00015A0D8EF11F01B5E18501C5ADBEF11F08E
:1023B0001B2618501C22153615341B361C36175098
:1023C00015A0E8EF11F01B5E18501C5AEBEF11F04E
:1023D0001B2618501C22153615341B361C36175078
:1023E00015A0F8EF11F01B5E18501C5AFBEF11F00E
:1023F0001B2618501C22153614341B361C36175059
:1024000015A008EF12F01B5E18501C5A0BEF12F0CB
:102410001B2618501C22143614341B361C36175039
:1024200014A018EF12F01B5E18501C5A1BEF12F08C
:102430001B2618501C22143614341B361C36175019
:1024400014A028EF12F01B5E18501C5A2BEF12F04C
:102450001B2618501C22143614341B361C361750F9
:1024600014A038EF12F01B5E18501C5A3BEF12F00C
:102470001B2618501C22143614341B361C361750D9
:1024800014A048EF12F01B5E18501C5A4BEF12F0CC
:102490001B2618501C22143614341B361C361750B9
:1024A00014A058EF12F01B5E18501C5A5BEF12F08C
:1024B0001B2618501C22143614341B361C36175099
:1024C00014A068EF12F01B5E18501C5A6BEF12F04C
:1024D0001B2618501C22143614341B361C36175079
:1024E00014A078EF12F01B5E18501C5A7BEF12F00C
:1024F0001B2618501C22143613341B361C3617505A
:1025000014A088EF12F01B5E18501C5A8BEF12F0CB
:102510001B2618501C22133613341B361C3617503A
:1025200013A098EF12F01B5E18501C5A9BEF12F08C
:102530001B2618501C22133613341B361C3617501A
:1025400013A0A8EF12F01B5E18501C5AABEF12F04C
:102550001B2618501C22133613341B361C361750FA
:1025600013A0B8EF12F01B5E18501C5ABBEF12F00C
:102570001B2618501C22133613341B361C361750DA
:1025800013A0C8EF12F01B5E18501C5ACBEF12F0CC
:102590001B2618501C22133613341B361C361750BA
:1025A00013A0D8EF12F01B5E18501C5ADBEF12F08C
:1025B0001B2618501C22133613341B361C3617509A
:1025C00013A0E8EF12F01B5E18501C5AEBEF12F04C
:1025D0001B2618501C22133613341B361C3617507A
:1025E00013A0F8EF12F01B5E18501C5AFBEF12F00C
:1025F0001B2618501C22133613B003EF13F017508C
:102600001B2618501C22A4B138EF13F024AE000C86
:10261000131E141E151E000E132A142215221B1E33
:102620001C1E1B2A1C22000C18AE32EF13F015BE24
:102630002DEF13F0E8CF9DF01450E8CF1CF01350AD
:10264000E8CF1BF01C9E143615361550E8CF13F05A
:102650009D51156A146A06EF13F0136A132A146A5F
:10266000156A000C151E141E131EA42B8FEF11F0FB
:102670001B2AE86A1C2217501B6206EF13F0185041
:102680001C6206EF13F01C6A1B6A000E132A142248
:10269000152215AE06EF13F02388FF0C1E6A1D6A83
:1026A0001C6A1B6A16341B361C361D361E36175024
:1026B0001B5E18501C5A19501D5A1A501E5AA46AF3
:1026C000A45B163616341B361C361D361E36A43750
:1026D000175016A077EF13F01B5E18501C5A1950B4
:1026E0001D5A1A501E5AE86AA45B80EF13F01B268D
:1026F00018501C2219501D221A501E22E86AA423C9
:10270000163616341B361C361D361E36A4371750A7
:1027100016A096EF13F01B5E18501C5A19501D5A44
:102720001A501E5AE86AA45B9FEF13F01B2618503C
:102730001C2219501D221A501E22E86AA4231636A4
:1027400016341B361C361D361E36A437175016A0FD
:10275000B5EF13F01B5E18501C5A19501D5A1A5031
:102760001E5AE86AA45BBEEF13F01B2618501C2209
:1027700019501D221A501E22E86AA4231636163458
:102780001B361C361D361E36A437175016A0D4EF44
:1027900013F01B5E18501C5A19501D5A1A501E5A1D
:1027A000E86AA45BDDEF13F01B2618501C221950B9
:1027B0001D221A501E22E86AA423163616341B3630
:1027C0001C361D361E36A437175016A0F3EF13F033
:1027D0001B5E18501C5A19501D5A1A501E5AE86A8E
:1027E000A45BFCEF13F01B2618501C2219501D226D
:1027F0001A501E22E86AA423163616341B361C36DD
:102800001D361E36A437175016A012EF14F01B5EAB
:1028100018501C5A19501D5A1A501E5AE86AA45BC7
:102820001BEF14F01B2618501C2219501D221A50A1
:102830001E22E86AA423163616341B361C361D36B3
:102840001E36A437175016A031EF14F01B5E185037
:102850001C5A19501D5A1A501E5AE86AA45B3AEFC6
:1028600014F01B2618501C2219501D221A501E222B
:10287000E86AA423163615341B361C361D361E3660
:10288000A437175016A050EF14F01B5E18501C5AB6
:1028900019501D5A1A501E5AE86AA45B59EF14F0D9
:1028A0001B2618501C2219501D221A501E22E86A9D
:1028B000A423153615341B361C361D361E36A43798
:1028C000175015A06FEF14F01B5E18501C5A1950CA
:1028D0001D5A1A501E5AE86AA45B78EF14F01B26A2
:1028E00018501C2219501D221A501E22E86AA423D7
:1028F000153615341B361C361D361E36A4371750B8
:1029000015A08EEF14F01B5E18501C5A19501D5A5A
:102910001A501E5AE86AA45B97EF14F01B26185051
:102920001C2219501D221A501E22E86AA4231536B3
:1029300015341B361C361D361E36A437175015A00D
:10294000ADEF14F01B5E18501C5A19501D5A1A5046
:102950001E5AE86AA45BB6EF14F01B2618501C221E
:1029600019501D221A501E22E86AA4231536153468
:102970001B361C361D361E36A437175015A0CCEF5B
:1029800014F01B5E18501C5A19501D5A1A501E5A2A
:10299000E86AA45BD5EF14F01B2618501C221950CE
:1029A0001D221A501E22E86AA423153615341B3640
:1029B0001C361D361E36A437175015A0EBEF14F049
:1029C0001B5E18501C5A19501D5A1A501E5AE86A9C
:1029D000A45BF4EF14F01B2618501C2219501D2282
:1029E0001A501E22E86AA423153615341B361C36ED
:1029F0001D361E36A437175015A00AEF15F01B5EC2
:102A000018501C5A19501D5A1A501E5AE86AA45BD5
:102A100013EF15F01B2618501C2219501D221A50B6
:102A20001E22E86AA423153615341B361C361D36C3
:102A30001E36A437175015A029EF15F01B5E18504D
:102A40001C5A19501D5A1A501E5AE86AA45B32EFDC
:102A500015F01B2618501C2219501D221A501E2238
:102A6000E86AA423153614341B361C361D361E3670
:102A7000A437175015A048EF15F01B5E18501C5ACC
:102A800019501D5A1A501E5AE86AA45B51EF15F0EE
:102A90001B2618501C2219501D221A501E22E86AAB
:102AA000A423143614341B361C361D361E36A437A8
:102AB000175014A067EF15F01B5E18501C5A1950E0
:102AC0001D5A1A501E5AE86AA45B70EF15F01B26B7
:102AD00018501C2219501D221A501E22E86AA423E5
:102AE000143614341B361C361D361E36A4371750C8
:102AF00014A086EF15F01B5E18501C5A19501D5A71
:102B00001A501E5AE86AA45B8FEF15F01B26185066
:102B10001C2219501D221A501E22E86AA4231436C2
:102B200014341B361C361D361E36A437175014A01D
:102B3000A5EF15F01B5E18501C5A19501D5A1A505B
:102B40001E5AE86AA45BAEEF15F01B2618501C2233
:102B500019501D221A501E22E86AA4231436143478
:102B60001B361C361D361E36A437175014A0C4EF72
:102B700015F01B5E18501C5A19501D5A1A501E5A37
:102B8000E86AA45BCDEF15F01B2618501C221950E3
:102B90001D221A501E22E86AA423143614341B3650
:102BA0001C361D361E36A437175014A0E3EF15F05F
:102BB0001B5E18501C5A19501D5A1A501E5AE86AAA
:102BC000A45BECEF15F01B2618501C2219501D2297
:102BD0001A501E22E86AA423143614341B361C36FD
:102BE0001D361E36A437175014A002EF16F01B5ED8
:102BF00018501C5A19501D5A1A501E5AE86AA45BE4
:102C00000BEF16F01B2618501C2219501D221A50CB
:102C10001E22E86AA423143614341B361C361D36D3
:102C20001E36A437175014A021EF16F01B5E185063
:102C30001C5A19501D5A1A501E5AE86AA45B2AEFF2
:102C400016F01B2618501C2219501D221A501E2245
:102C5000E86AA423143613341B361C361D361E3680
:102C6000A437175014A040EF16F01B5E18501C5AE2
:102C700019501D5A1A501E5AE86AA45B49EF16F003
:102C80001B2618501C2219501D221A501E22E86AB9
:102C9000A423133613341B361C361D361E36A437B8
:102CA000175013A05FEF16F01B5E18501C5A1950F6
:102CB0001D5A1A501E5AE86AA45B68EF16F01B26CC
:102CC00018501C2219501D221A501E22E86AA423F3
:102CD000133613341B361C361D361E36A4371750D8
:102CE00013A07EEF16F01B5E18501C5A19501D5A87
:102CF0001A501E5AE86AA45B87EF16F01B2618507C
:102D00001C2219501D221A501E22E86AA4231336D1
:102D100013341B361C361D361E36A437175013A02D
:102D20009DEF16F01B5E18501C5A19501D5A1A5070
:102D30001E5AE86AA45BA6EF16F01B2618501C2248
:102D400019501D221A501E22E86AA4231336133488
:102D50001B361C361D361E36A437175013A0BCEF89
:102D600016F01B5E18501C5A19501D5A1A501E5A44
:102D7000E86AA45BC5EF16F01B2618501C221950F8
:102D80001D221A501E22E86AA423133613341B3660
:102D90001C361D361E36A437175013A0DBEF16F075
:102DA0001B5E18501C5A19501D5A1A501E5AE86AB8
:102DB000A45BE4EF16F01B2618501C2219501D22AC
:102DC0001A501E22E86AA423133613341B361C360D
:102DD0001D361E36A437175013A0FAEF16F01B5EEF
:102DE00018501C5A19501D5A1A501E5AE86AA45BF2
:102DF00003EF17F01B2618501C2219501D221A50E1
:102E00001E22E86AA423133613341B361C361D36E3
:102E10001E36A437175013A019EF17F01B5E185079
:102E20001C5A19501D5A1A501E5AE86AA45B22EF08
:102E300017F01B2618501C2219501D221A501E2252
:102E4000E86AA423133613B02EEF17F017501B2691
:102E500018501C2219501D221A501E22000C0F015E
:102E6000D89083B6D880D8B03BEF17F00A0E9DEC0F
:102E70000BF00F01D89083B6D880D8B0B1EF17F01F
:102E80000F01D89084B2D880D8B04CEF17F00A0E5A
:102E90009DEC0BF00F01D89084B2D880D8B0B1EF80
:102EA00017F00001CC6773EF17F00001CC69030144
:102EB00032C30DF033C30EF00001E80E0F6E030EA7
:102EC000106E67EC10F014C01CF115C01DF1030169
:102ED000345101011C270301355101011D2334C365
:102EE0001AF135C31BF1A8EC29F0D8B084EF17F024
:102EF000D8A48BEF17F001011A07D8A01B071A07F7
:102F0000D8A01B078BEF17F001011A2BD8B41B2B8D
:102F10001A2BD8B41B2B1CC10DF01DC10EF00101E2
:102F20001A5100010D5E01011B5100010E5A0001F2
:102F3000000E0F6E010E106E67EC10F00001E80E2F
:102F4000176E030E186E6BEC11F013C032F314C041
:102F500033F31AC134F31BC135F311EC1AF0D884E2
:102F600012000001CC67B7EF17F0D8941200CC6BB9
:102F700084EC1FF0D894120000016951E8CF0DF0E5
:102F80006A51E8CF0EF06D510D5E6E510E5AD8A009
:102F9000D9EF17F06B51E8CF0FF06C51E8CF10F07C
:102FA00067EC10F01450E8CF71F01550E8CF72F0D4
:102FB00012006F51E8CF0FF07051E8CF10F067ECBE
:102FC00010F01450E8CF71F01550E8CF72F01200F5
:102FD00069C00DF06AC00EF06D510D5E6E510E5A53
:102FE0006BC00FF06CC010F067EC10F01450E8CF1D
:102FF00071F01550E8CF72F01200040E93EC08F057
:10300000040EBBEC08F015C26BF016C26CF017C2D0
:103010006DF018C26EF019C26FF01AC270F0BCECFD
:1030200017F071C034F172C035F171C073F072C025
:1030300074F0050E93EC08F0050EBBEC08F01BC213
:103040006BF01CC26CF01DC26DF01EC26EF01FC290
:103050006FF020C270F0BCEC17F071C036F172C096
:1030600037F171C075F072C076F0060E93EC08F07F
:10307000060EBBEC08F021C26BF022C26CF023C23A
:103080006DF024C26EF025C26FF026C270F0BCEC69
:1030900017F071C038F172C039F171C077F072C0A9
:1030A00078F0070E93EC08F0070E93EC08F027C2B7
:1030B0006BF028C26CF029C26DF02AC26EF0E8EC09
:1030C00017F071C03AF172C03BF171C079F072C073
:1030D0007AF0030E93EC08F000010F01C3CFE8FF74
:1030E000E8CF8BF0C4CFE8FFE8CF8CF0080E93EC6C
:1030F00008F02DC26DF02EC26EF02BC26BF02CC208
:103100006CF0E8EC17F071C083F072C084F0090E27
:1031100093EC08F031C26DF032C26EF02FC26BF04A
:1031200030C26CF0E8EC17F071C085F072C086F028
:103130000A0E93EC08F035C26DF036C26EF033C261
:103140006BF034C26CF0E8EC17F071C087F072C01D
:1031500088F00B0E93EC08F039C26DF03AC26EF0B5
:1031600037C26BF038C26CF0E8EC17F071C089F030
:1031700072C08AF00301B5517FEC24F0D8A0C7EFEC
:1031800018F0030E7C6FE80E7B6FC9EF18F07B6BB5
:103190007C6B000E93EC08F03BC26BF03CC26CF011
:1031A0003DC26DF03EC26EF0E8EC17F071C07DF0EC
:1031B00072C07EF0010E93EC08F03FC26BF040C28B
:1031C0006CF041C26DF042C26EF0E8EC17F071C0D5
:1031D0007FF072C080F00301B7517FEC24F0D8A0DB
:1031E000F8EF18F0030E826FE80E816F0EEF19F002
:1031F0000301B9517FEC24F0D8A003EF19F0816BE3
:10320000826B0EEF19F00301B8517FEC24F0D8A0C7
:103210000EEF19F0010E826FF40E816F12000001A3
:10322000106A0FBE101E67EC10F00001640E176EDE
:10323000000E186E6BEC11F013C011F014C012F0F8
:1032400013C00FF014C010F00EAE2CEF19F00F1ECB
:10325000101E0F2AD8B0102A67EC10F000010A0ED9
:10326000176E000E186E6BEC11F00B50E8CF17F0D4
:10327000186A17BE181E6BEC11F011500D5E12503B
:103280000E5A13500D2614500E2212000301AE5197
:103290007FEC24F073C00DF074C00EF0D8A05CEF8A
:1032A00019F003011B510001E8CF0FF00301175182
:1032B000E8CF0BF064EF19F003011A510001E8CFD9
:1032C0000FF0640EE8CF0BF00FEC19F00DC073F0A7
:1032D0000EC074F00301AF517FEC24F075C00DF007
:1032E00076C00EF0D8A080EF19F00301265100013E
:1032F000E8CF0FF003012251E8CF0BF088EF19F06F
:10330000030125510001E8CF0FF0640EE8CF0BF068
:103310000FEC19F00DC075F00EC076F00301B0513E
:103320007FEC24F077C00DF078C00EF0D8A0A4EFA9
:1033300019F0030131510001E8CF0FF003012D51C5
:10334000E8CF0BF0ACEF19F0030130510001E8CFEA
:103350000FF0640EE8CF0BF00FEC19F00DC077F012
:103360000EC078F012000301AE517FEC24F0D8A01B
:10337000D2EF19F073C00FF074C010F017C30DF046
:1033800018C30EF00E6A0DBE0E1E67EC10F00001A1
:10339000640E176E000E186E6BEC11F013C073F014
:1033A00014C074F00301AF517FEC24F0D8A0F1EF0A
:1033B00019F075C00FF076C010F022C30DF023C3D2
:1033C0000EF00E6A0DBE0E1E67EC10F00001640ECA
:1033D000176E000E186E6BEC11F013C075F014C070
:1033E00076F00301B0517FEC24F0D8A010EF1AF072
:1033F00077C00FF078C010F02DC30DF02EC30EF083
:103400000E6A0DBE0E1E67EC10F00001640E176E02
:10341000000E186E6BEC11F013C077F014C078F04A
:1034200012000201B2519BEC01F00301A75100010F
:103430000F260301A8510001102218C30DF019C373
:103440000EF000010E6AFF0E0DBE0E6E67EC10F05E
:103450000001640E176E186A196A1A6A6BEC11F093
:1034600000010301195100010D6E0E6A0DBE0E1E02
:103470000D360E360D5013260E501422135073279E
:10348000145074230201B3519BEC01F00301A951C4
:1034900000010F260301AA510001102223C30DF0E1
:1034A00024C30EF000010E6AFF0E0DBE0E6E67EC17
:1034B00010F00001640E176E186A196A1A6A6BEC34
:1034C00011F000010301245100010D6E0E6A0DBEC2
:1034D0000E1E0D360E360D5013260E5014221350AC
:1034E0007527145076230201B4519BEC01F00301BF
:1034F000AB5100010F260301AC51000110222EC375
:103500000DF02FC30EF000010E6AFF0E0DBE0E6E01
:1035100067EC10F00001640E176E186A196A1A6AD7
:103520006BEC11F0000103012F5100010D6E0E6ACA
:103530000DBE0E1E0D360E360D5013260E501422E3
:1035400013507727145078230201B5519BEC01F0FA
:1035500036C30DF037C30EF000010E6AFF0E0DBE2C
:103560000E6E67EC10F00001640E176E186A196A8F
:103570001A6A6BEC11F00301010E3763D7EF1AF0F2
:103580000001030E0E6E186EE80E0D6E176E795167
:103590000D5E7A510E5A196A1A6A13C00FF014C0E0
:1035A00010F067EC10F06BEC11F0F1EF1AF0020E76
:1035B0003763F1EF1AF0000179510D6E7A510E6EFA
:1035C00013C00FF014C010F067EC10F00001030EF0
:1035D000E8CF18F0E80EE8CF17F0196A1A6A6BEC1A
:1035E00011F000011350792714507A2312000001C2
:1035F0000E6A08C40DF00DBE0E6800010A0E0F6EB3
:10360000000E106E67EC10F01350732714507423E3
:1036100000010E6A09C40DF00DBE0E6800010A0E0D
:103620000F6E000E106E67EC10F0135075271450DB
:10363000762300010E6A0AC40DF00DBE0E6800016B
:103640000A0E0F6E000E106E67EC10F01350772705
:103650001450782300010E6A0BC40DF00DBE0E68E5
:1036600000010A0E0F6E000E106E67EC10F0135082
:10367000792714507A2300010E6A0CC40DF00DBE98
:103680000E6800010A0E0F6E000E106E67EC10F04F
:1036900013507B2714507C2300010E6A0DC40DF0DB
:1036A0000DBE0E6800010A0E0F6E000E106E67EC64
:1036B00010F013507D2714507E2300010E6A0EC4B3
:1036C0000DF00DBE0E6800010A0E0F6E000E106E9A
:1036D00067EC10F013507F271450802300010E6A0E
:1036E0000FC40DF00DBE0E6800010A0E0F6E000E25
:1036F000106E67EC10F013508127145082231200D3
:1037000000010A0E0D6E000E0E6E0301BB517FEC20
:1037100024F0D8A0C8EF1BF003014DAF9BEF1BF0C6
:103720004CC30FF0106A0FBE106867EC10F013C0A6
:1037300073F014C074F003014FAFAAEF1BF04EC337
:103740000FF0106A0FBE106867EC10F013C075F030
:1037500014C076F0030151AFB9EF1BF050C30FF066
:10376000106A0FBE106867EC10F013C077F014C039
:1037700078F0030153AFC8EF1BF052C30FF0106A8B
:103780000FBE106867EC10F013C079F014C07AF027
:103790000301BC517FEC24F0D8A00BEF1CF0030117
:1037A00055AFDEEF1BF054C30FF0106A0FBE106868
:1037B00067EC10F013C073F014C074F0030157AF3E
:1037C000EDEF1BF056C30FF0106A0FBE106867ECE8
:1037D00010F013C075F014C076F0030159AFFCEF80
:1037E0001BF058C30FF0106A0FBE106867EC10F0A2
:1037F00013C077F014C078F003015BAF0BEF1CF03F
:103800005AC30FF0106A0FBE106867EC10F013C0B7
:1038100079F014C07AF000017AAF1200E86A796F8B
:103820007A6F12000201A1B112000301B6517FECC0
:1038300024F0D8A0120000016067120002019F511D
:103840000001606F0201010EB66330EF1CF0010E43
:1038500000015D6E050E37EC0AF0280E0001606F66
:1038600073C00DF074C00EF0D3EC1CF0D8A466EF5A
:103870001CF00201B6673FEF1CF002019E510001EF
:1038800074BF4DEF1CF00301192719AF57EF1CF05F
:10389000D8A657EF1CF05AEF1CF00301195F19BFAF
:1038A00057EF1CF0D8A657EF1CF05FEF1CF019BFC4
:1038B0005FEF1CF0640E1961196F64EF1CF0640E69
:1038C000E81EE82A1965196F84EC1FF075C00DF029
:1038D00076C00EF0D3EC1CF0D8A49CEF1CF00201D3
:1038E000B66775EF1CF002019E51000176BF83EFB1
:1038F0001CF00301242724AF8DEF1CF0D8A68DEF18
:103900001CF090EF1CF00301245F24BF8DEF1CF02E
:10391000D8A68DEF1CF095EF1CF024BF95EF1CF09E
:10392000640E2461246F9AEF1CF0640EE81EE82AEE
:103930002465246F84EC1FF077C00DF078C00EF082
:10394000D3EC1CF0D8A4D2EF1CF00201B667ABEFA9
:103950001CF002019E51000178BFB9EF1CF0030179
:103960002F272FAFC3EF1CF0D8A6C3EF1CF0C6EF74
:103970001CF003012F5F2FBFC3EF1CF0D8A6C3EFCD
:103980001CF0CBEF1CF02FBFCBEF1CF0640E2F61AF
:103990002F6FD0EF1CF0640EE81EE82A2F652F6F02
:1039A00084EC1FF0120000010EAEDCEF1CF00D1EC7
:1039B0000E1E0D2AD8B00E2AD8900E320D320E6689
:1039C000E6EF1CF0640E0D64EBEF1CF00001640EDA
:1039D0000D6E000E0E6E0D50E832E8321F0BD874DB
:1039E0000DC0E8FF12000001BD6B000174BF05EFC0
:1039F0001DF011C30DF012C30EF073C00FF074C0B0
:103A000010F067EC10F00FEF1DF015C30DF016C3AA
:103A10000EF073C00FF074C010F067EC10F013C319
:103A20000DF014C30EF0000114500D2615500E2297
:103A300064EC1EF00DC03CF00EC03DF0000176BFFE
:103A40002EEF1DF01CC30DF01DC30EF075C00FF05E
:103A500076C010F067EC10F038EF1DF020C30DF0C9
:103A600021C30EF075C00FF076C010F067EC10F0B7
:103A70001EC30DF01FC30EF0000114500D2615508B
:103A80000E2264EC1EF00DC03AF00EC03BF00001B7
:103A900078BF57EF1DF027C30DF028C30EF077C095
:103AA0000FF078C010F067EC10F061EF1DF02BC341
:103AB0000DF02CC30EF077C00FF078C010F067EC5B
:103AC00010F029C30DF02AC30EF0000114500D268A
:103AD00015500E2264EC1EF00DC03EF00EC03FF0FB
:103AE00032C30DF033C30EF079C00FF07AC010F07E
:103AF00067EC10F034C30DF035C30EF00001145024
:103B00000D2615500E2264EC1EF00DC040F00EC0C4
:103B100041F03AC30DF03BC30EF07BC00FF07CC008
:103B200010F067EC10F03CC30DF03DC30EF0000147
:103B300014500D2615500E2264EC1EF00DC042F0FC
:103B40000EC043F0040117A1CBEF1DF000017EBFB2
:103B5000B6EF1DF01CC30DF01DC30EF07DC00FF0BD
:103B60007EC010F067EC10F0C0EF1DF020C30DF028
:103B700021C30EF07DC00FF07EC010F067EC10F096
:103B80001EC30DF01FC30EF0000114500D2615507A
:103B90000E22DEEF1DF03EC30DF03FC30EF07DC0E0
:103BA0000FF07EC010F067EC10F040C30DF041C381
:103BB0000EF0000114500D2615500E2264EC1EF07C
:103BC0000DC044F00EC045F003019AA10DEF1EF0A8
:103BD000000180BFF8EF1DF011C30DF012C30EF00D
:103BE0007FC00FF080C010F067EC10F002EF1EF005
:103BF00015C30DF016C30EF07FC00FF080C010F09B
:103C000067EC10F013C30DF014C30EF00001145054
:103C10000D2615500E2220EF1EF042C30DF043C3B7
:103C20000EF07FC00FF080C010F067EC10F044C3BE
:103C30000DF045C30EF0000114500D2615500E2254
:103C400064EC1EF00DC046F00EC047F081C00DF0D0
:103C500082C00EF0F40E0D5E010E0E5AD8900D3695
:103C60000E360EBE3CEF1EF046C30FF047C310F0F9
:103C700067EC10F042EF1EF04AC30FF04BC310F098
:103C800067EC10F048C30DF049C30EF00D50142638
:103C90000E50152214C00DF015C00EF064EC1EF08D
:103CA0000DC048F00EC049F00001CC6763EF1EF074
:103CB0000301B1517FEC24F0D8A063EF1EF038C3AC
:103CC00040F039C341F012000201AE5100010D5C19
:103CD0000201AF5100010E58E8AE74EF1EF0AEC203
:103CE0000DF0AFC20EF012000201B05100010D5CE8
:103CF0000201B15100010E58E8BE1200B0C20DF031
:103D0000B1C20EF01200000133B492EF1EF035A4E0
:103D100092EF1EF03594010E5D6E050E37EC0AF041
:103D2000D8801200D89012000001000E0D6E020E15
:103D30000E6E0001000E136E000E146E010E156E55
:103D4000E86A0A6E10EC0CF0020100510001A56F48
:103D500012000001000E0D6E020E0E6E0001000E2C
:103D6000136E000E146E010E156E040E0A6E44ECF6
:103D70000CF01200E846E8060B6E0001000E0D6E16
:103D8000030E0E6E0001000E136E000E146E010E77
:103D9000156E0B501426E86A1522100E0A6E10ECF0
:103DA0000CF01200E846E8060B6E0001000E0D6EE6
:103DB000080E0E6E0001000E136E000E146E010E42
:103DC000156E0B501426E86A1522400E0A6E10EC90
:103DD0000CF00001000EB56F030EB66F0001000E6F
:103DE000B36F030EB46F0001080EB46F100EB76FFF
:103DF00057EC23F00001000E0D6E080E0E6E000150
:103E0000000E136E000E146E010E156E0B5014266C
:103E1000E86A1522010E0A6E44EC0CF01200E84626
:103E2000E8060B6E0001000E0D6E030E0E6E000113
:103E3000000E136E000E146E010E156E0B5014263C
:103E4000E86A15220A6E10EC0CF00001000E0D6EEF
:103E5000040E0E6E0001000E136E000E146E010EA5
:103E6000156E0B50E82A1426E86A15220A6E10EC2B
:103E70000CF01200E846E8060C6E0001000E0D6E14
:103E8000030E0E6E0001000E136E000E146E010E76
:103E9000156E0C501426E86A1522040E0A6E44ECC6
:103EA0000CF00001000E0D6E040E0E6E0001000EEF
:103EB000136E000E146E010E156E0C50E82A1426B7
:103EC000E86A1522040E0A6E44EC0CF012000001A0
:103ED000000EB56F030EB66F0001000EB36F060E35
:103EE000B46F000EB76F57EC23F00001000EB56FF2
:103EF000040EB66F0001000EB36F070EB46F000E14
:103F0000B76F57EC23F0120002010051E846E806B3
:103F10000A6E0001000E0D6E030E0E6E0001000E03
:103F2000136E000E146E010E156E0A501426E86A08
:103F30001522010E0A6E44EC0CF0120073C08DF0D5
:103F400074C08EF075C08FF076C090F077C091F09D
:103F500078C092F079C093F07AC094F07BC095F06D
:103F60007CC096F07DC097F07EC098F07FC099F03D
:103F700080C09AF081C09BF082C09CF012009EEC41
:103F80001FF00301B2517FEC24F0D8B0DAEF1FF03C
:103F9000030EE26E5C0EE16E77EC22F0610EE16ED4
:103FA00077EC22F0660EE16E77EC22F06B0EE16E9C
:103FB00077EC22F09EEC1FF00301B3517FEC24F06C
:103FC000D8B0FBEF1FF0030EE26E700EE16E77ECDF
:103FD00022F09EEC1FF0750EE16E77EC22F09EEC65
:103FE0001FF07A0EE16E77EC22F09EEC1FF07F0E50
:103FF000E16E77EC22F09EEC1FF00301B4517FECF0
:1040000024F0D8B016EF20F0030EE26E840EE16EBD
:1040100077EC22F0890EE16E77EC22F08E0EE16EE5
:1040200077EC22F0930EE16E77EC22F012008DC057
:104030000DF08EC00EF010C40FF000010EBE11C4C2
:104040000FF0106A0FBE106867EC10F00001640EEC
:10405000176E000E186E6BEC11F0000113C0E8FF34
:10406000912714C0E8FF922391C00DF092C00EF08A
:1040700012C40FF000010EBE13C40FF0106A0FBE81
:10408000106867EC10F00001640E176E000E186ED9
:104090006BEC11F0000113C0E8FF8D2714C0E8FF9E
:1040A0008E2391C00DF092C00EF014C40FF00001E9
:1040B0000EBE15C40FF0106A0FBE106867EC10F04A
:1040C0000001640E176E000E186E6BEC11F000010B
:1040D00013C0E8FF8F2714C0E8FF902393C00DF0B2
:1040E00094C00EF016C40FF000010EBE106A0FBE91
:1040F000106867EC10F00001640E176E000E186E69
:104100006BEC11F0000113C0E8FF8F2714C0E8FF2B
:1041100090238DC073F08EC074F08FC075F090C086
:1041200076F091C077F092C078F093C079F094C0A7
:104130007AF0040117A1ABEF20F08FC07DF090C0A2
:104140007EF0040118A1ABEF20F000017D1F7E1F5F
:104150007D2BD8B07E2B030198A1C8EF20F08FC033
:104160000DF090C00EF091C00FF092C010F0000161
:104170000DC075F00EC076F00DC077F00EC078F06F
:104180000F507727105078230F50755F1050765BD3
:10419000030199A1E5EF20F08FC00DF090C00EF063
:1041A0008DC00FF08EC010F000010DC075F00EC074
:1041B00076F00DC073F00EC074F00F5073271050DE
:1041C00074230F50755F1050765B03019AA19FEF27
:1041D00021F08DC00DF08EC00EF00DC073F00EC03A
:1041E00074F00DC07FF00EC080F00001640E176EF9
:1041F000000E186E03019C51E812D8B44BEF21F069
:10420000E8BE28EF21F0640800010F6E106A74BF49
:1042100016EF21F073C00DF074C00EF067EC10F0D3
:104220006BEC11F013C073F014C074F0000180AF98
:104230004BEF21F07FC00DF080C00EF067EC10F066
:104240006BEC11F013C07FF014C080F04BEF21F045
:10425000640F00010F6E106A74AF3BEF21F073C062
:104260000DF074C00EF067EC10F06BEC11F013C0A1
:1042700073F014C074F0000180BF4BEF21F07FC0D9
:104280000DF080C00EF067EC10F06BEC11F013C075
:104290007FF014C080F003019BA155EF21F00001D5
:1042A0007F1F801F7F2BD8B0802B0001640E176EFC
:1042B000000E186E03019D51E812D8B49FEF21F053
:1042C0000301C651E812D8B478EF21F00301C551BB
:1042D0007FEC24F0D8B09FEF21F00001E80E0D6EC6
:1042E000030E0E6E93510D5E94510E5A81EF21F024
:1042F0000001E80E0D6E030E0E6E99510D5E9A517F
:104300000E5A9DC30FF09EC310F0106AE8BE101E37
:1043100067EC10F06BEC11F01350732714507423FA
:1043200003019BB19AEF21F00001131E141E132A02
:10433000D8B0142A000113507F2714508023120094
:104340000301A4A112009EEC1FF017EC20F0120054
:104350000301A4B1B0EF21F09EEC1FF017EC20F0A8
:1043600003019EA1CBEF21F00301C2517FEC24F0A9
:10437000D8A0CBEF21F003019F5100010D6E0E6A12
:1043800000010A0E0F6E000E106E67EC10F013C0E5
:1043900079F014C07AF00301A0A1F8EF21F0030135
:1043A000C3517FEC24F0D8A0DAEF21F00301A15132
:1043B000E3EF21F00301C4517FEC24F0D8A0F8EF23
:1043C00021F00301A25100010D6E0E6A00010A0ED8
:1043D0000F6E000E106E67EC10F01350795D1450E4
:1043E0007A59E8AEF8EF21F013C079F014C07AF0F2
:1043F00012000BC0E8FFF00BD8B412000DC069F03A
:104400000EC06AF00EAE0AEF22F00D1E0E1E0D2A2F
:10441000D8B00E2A0DC013F00EC014F0640E176E43
:104420009AEC10F000011C6A090E136022EF22F0D2
:104430000BC0E8FFE83AE8060F0BE8B63FEF22F0C2
:1044400034EF22F0136E0DC01BF00EC01CF0840E72
:1044500000011B5E030E1C5A0BC0E8FFE83AE80699
:104460000F0BE8B63FEF22F00B0DF350460F13246D
:10447000E8CFD9FF020EE8CFDAFF49EF22F0E89645
:104480000B0DF350DA0F1324E8CFD9FF030EE8CF5A
:10449000DAFFDECF0AF0DFCF0BF000010BC00DF02A
:1044A0000AC0E8FF0D5E0E6A0DBE0E681BC00FF05D
:1044B0001CC010F067EC10F00A0E176E9AEC10F0AA
:1044C0000AC0E8FF0A0DF3CFE8FF1326F4CFE8FF98
:1044D000142213C00DF014C00EF000016AAF1200D8
:1044E00000010D1E0E1E0D2AD8B00E2A1200E65035
:1044F000E8CF0BF0E812D8B4120080EC02F0F9EC2F
:1045000021F00DC011F00EC012F0E6CF0AF0E6CF98
:10451000E8FF0001E8CF0DF00E6A0DBE0E1E00018F
:104520000A0E0F6E000E106E67EC10F011C00DF049
:1045300012C00EF013500D5E14500E5A0EBED6EF80
:1045400022F0E6CFE8FF00010AACBFEF22F0E8CF8F
:1045500013F0E9CF14F00DC011F00EC012F013509B
:1045600080EC02F00DC013F00EC014F00A0E176EAE
:104570009AEC10F011C00DF012C00EF013500F6E37
:10458000106A0FBE101E67EC10F00001640E176E6B
:10459000000E186E196A1A6A6BEC11F013C00DF058
:1045A00014C00EF00A5000EC03F01200E6CFE8FF52
:1045B000E6CFE8FF00010AAAF4EF22F0E8CF13F0FB
:1045C0000DC011F00EC012F0135080EC02F00DC0BF
:1045D00013F00EC014F00A0E176E9AEC10F011C012
:1045E0000DF012C00EF013500F6E106A0FBE101EA9
:1045F00067EC10F00001640E176E000E186E196A59
:104600001A6A6BEC11F013C00DF014C00EF00A50D2
:1046100000EC03F012000001BD0EB56F030EB66F83
:104620000001120EB36F010EB46F050EB76F57EC99
:1046300023F0D90EE8CFD9FF060EE8CFDAFF060E39
:10464000E8CF0CF0DDCFE8FFE812D8B42FEF23F06D
:10465000DFCFE8FF7FEC24F0D8B03BEF23F0DDCFD5
:10466000E8FF0C2E22EF23F0A5C0E8FF0201006353
:1046700044EF23F01200DECFE8FFDECFE8FF0201B7
:10468000006344EF23F01200E8CF00F20FEC1FF0BC
:104690000001120EB56F010EB66F0001BD0EB36FB3
:1046A000030EB46F050EB76F57EC23F01200000134
:1046B000B551E16EB651E26E0001B351D96EB451FD
:1046C000DA6EE6CFE8FFE8CFDEFF0001B72F61EF3B
:1046D00023F012000001BF6B0301AE517FEC24F008
:1046E0000001D8B0BF810301AF517FEC24F000017D
:1046F000D8B0BF830301B0517FEC24F00001D8B0E3
:10470000BF850301B1517FEC24F00001D8B0BF8711
:104710000301B6517FEC24F00001D8B0BF8903013A
:10472000BB517FEC24F00001D8B0BF8B0301BC511A
:104730007FEC24F00001D8B0BF8D1200C00E0FEC4A
:104740000DF00301AE517FEC24F00001E86AE8802F
:10475000BF15D8A0BAEF23F0D8A4CBEF23F0BF71D8
:10476000000EF86E650EF76E220EF66E85EC0DF0FB
:104770007CEF24F0D8B0CBEF23F0D8B4CBEF23F00C
:10478000BF71000EF86E650EF76E100EF66E85ECBA
:104790000DF07CEF24F00301AF517FEC24F0000119
:1047A000E86AE882BF15D8A0E4EF23F0D8A4F5EFBB
:1047B00023F0BF73000EF86E650EF76E460EF66EB0
:1047C00085EC0DF07CEF24F0D8B0F5EF23F0D8B4F1
:1047D000F5EF23F0BF73000EF86E650EF76E340E22
:1047E000F66E85EC0DF07CEF24F00301B0517FEC08
:1047F00024F00001E86AE884BF15D8A00EEF24F089
:10480000D8A41FEF24F0BF75000EF86E650EF76E8A
:104810006A0EF66E85EC0DF07CEF24F0D8B01FEF39
:1048200024F0D8B41FEF24F0BF75000EF86E650EAB
:10483000F76E580EF66E85EC0DF07CEF24F0030158
:10484000B1517FEC24F00001D8A035EF24F0BFB7C0
:1048500036EF24F0BF77000EF86E650EF76EB20EDD
:10486000F66E85EC0DF07CEF24F0BF970301B65196
:104870007FEC24F00001D8A04CEF24F0BFB94DEF3D
:1048800024F0BF79000EF86E650EF76EA00EF66E7E
:1048900085EC0DF07CEF24F0BF990301BB517FEC58
:1048A00024F00001D8A063EF24F0BFBB64EF24F034
:1048B000BF7B000EF86E650EF76E7C0EF66E85EC13
:1048C0000DF07CEF24F0BF9B0301BC517FEC24F082
:1048D0000001D8A07AEF24F0BFBD7BEF24F0BF7DAC
:1048E000000EF86E650EF76E8E0EF66E85EC0DF00E
:1048F0007CEF24F0BF9D1200500EA36F1200E8AAB7
:10490000ABEF24F0E8A8ABEF24F00A6E070BC90F59
:10491000E16E030EE26EE65000010D6E0E6AE8BE17
:104920000E6800010A0E0F6E000E106E67EC10F09C
:104930000A50070BE846340FE16E010EE252E650D2
:10494000E6CF0BF00001135E0B501458E8360ABE98
:104950001200D8701200D890E8BA1200D880E8B8D7
:10496000120000011F6E206AE8BC2080070BE82AB5
:10497000D8802036E82EB9EF24F030501FB63350DF
:104980002014D8802062D8901FBED8701200040E68
:10499000D56E1200D59E1200D89087B21200D88032
:1049A000D5BE1200C3C00DF0C4C00EF000013C0E15
:1049B0000F6E000E106E78EC10F013C00DF014C0E6
:1049C0000EF00001240E0F6EF40E106E78EC10F055
:1049D000C1C017F0C2C018F00001000E196E000E21
:1049E0001A6E4EEC13F0A5C317F0A6C318F0000121
:1049F000186A6BEC11F0C00E0FEC0DF0000EF86EA3
:104A0000640EF76E800EF66E85EC0DF0CB0E0FEC9B
:104A10000DF0EBEC0DF0A5C313F0A6C314F0146A6F
:104A2000C00E0FEC0DF0E7EC0DF00001000EC36FAF
:104A3000000EC46FD88012000001020E3662120010
:104A4000000133A01200FC6A0AEF05F035EC25F0F6
:104A5000D8A01200FC6AA9EC1EF000C2E8FF3AECF4
:104A60001FF067EC1FF00AEF05F0000130B63FEFD2
:104A700025F032A63FEF25F03296D8801200D8906C
:104A800012000001650E0E6ED60E0D6E80EC25F044
:104A900064EC0DF00001115080EC01F012001EC119
:104AA0000DF01FC10EF064EC0DF012000001EF518B
:104AB000D8B41200FDEC17F00001000E736F000E69
:104AC000746F0001000E756F000E766FB3EC19F075
:104AD00046EC19F080EC1BF012EC1CF011EC1AF013
:104AE000A0EC21F0BFEC1FF0A8EC21F0F7EC1AF0DD
:104AF000F3EC1CF05EEC0EF012000001EF69120006
:104B00001CEC25F00001CD6BDB6BEA6BEB6BC00E90
:104B10000FEC0DF00DC0F6FF0EC0F7FFF86A0DC0E8
:104B20000FF00EC010F085EC0DF0FA0E9DEC0BF0BE
:104B300082EC29F0D8A4A3EF25F0110E0D26D8B0F1
:104B40000E2AAAEF25F0D8A0B7EF25F0130E0D26F8
:104B5000D8B00E2A0DC0F6FF0EC0F7FFF86A0900A4
:104B6000F5CF0DF00900F5CF0EF087EF25F026EC1C
:104B700025F083EC1EF0D8A087EF25F0150E0D264A
:104B8000D8B00E2A0DC0F6FF0EC0F7FFF86A090074
:104B9000F5CF11F00900F5CF12F00FC00DF010C0E5
:104BA0000EF00900F5CF0FF00900F5CF10F0090065
:104BB000F5CFCEF00900F5CFCFF00001B96BBA6B9D
:104BC000BB697F0EE8CFBCF012ACF3EF25F0090013
:104BD000F5CFB9F00900F5CFBAF00900F5CFBBF079
:104BE0000900F5CFBCF012A4FCEF25F00900F5CFC9
:104BF000EAF00900F5CFEBF012A205EF26F009006C
:104C0000F5CFECF00900F5CFEDF012AE0AEF26F08B
:104C100064EC0DF012A60FEF26F07AEC0DF012A264
:104C200012000001E86AE8CFFBFFEDC0E8FFE8CF23
:104C3000FAFFECC0E8FFF96EE8CF0AF00FC01BF0F6
:104C400010C01CF00FC0F6FF10C0F7FFF86A150E79
:104C5000F626D8B0F72A0900F5CFE8FF0A6232EF4E
:104C600026F012000FC0F6FF10C0F7FF110EF62657
:104C7000D8B0F72A0900F5CF0FF00900F5CF10F0F2
:104C80000FC0E8FF1B6222EF26F010C0E8FF1C6295
:104C900022EF26F01200000110500F10D8B41200BD
:104CA000E86AFB6E1050E8CFFAFF0F50F96E000172
:104CB0000F50E16E1050E26E0001000E116275EFB0
:104CC00026F00FC0F6FF10C0F7FFF86A160EF626A2
:104CD000D8B0F72ACEC0E1FFCFC0E2FFE7CFE8FFB0
:104CE0001CEC26F0EFEC28F01200010E11627CEFB4
:104CF00026F01EEC28F01200020E1162A6EF26F03C
:104D0000000112A087EF26F0CE510001B86FE6CF68
:104D10000AF0E5CF0BF000010AC011F00BC012F051
:104D2000129E129C74EC28F000010FC0E1FF10C02D
:104D3000E2FF11C00AF012C00BF00AC0E6FFE7CF95
:104D4000E8FFC00B0B120BC0E5FF1200030E11624F
:104D5000BBEF26F0E7CFE8FFE83677EC27F0000E50
:104D6000D8B0E81E0A6E00010FC0E1FF10C0E2FFDC
:104D70000AC0E7FF1200040E1162CCEF26F0E7CF65
:104D8000E8FF36EC29F00A6E00010FC0E1FF10C009
:104D9000E2FF0AC0E7FF1200050E1162DEEF26F007
:104DA000E7CFE8FFCCEC27F0E8CF0AF000010FC016
:104DB000E1FF10C0E2FF0AC0E7FF1200060E116219
:104DC000F4EF26F0E7CF0AF00FC0CEF010C0CFF01E
:104DD00000018A0E0F6E790E106E0AC0E8FF1CECFF
:104DE00026F0EFEC28F01200070E1162FBEF26F020
:104DF0004BEC26F01200080E11620CEF27F0E7CF03
:104E0000E8FFC6EC27F0E8CF0AF000010FC0E1FF91
:104E100010C0E2FF0AC0E7FF0A0E11622DEF27F073
:104E2000E7CFE8FF0001CE15D890D8B4D88077EC52
:104E300027F00001CEC00AF000010FC0E1FF10C052
:104E4000E2FFD8B028EF27F00AC0E8FFE71212000F
:104E50000AC0E8FFE81EE716120012000B6AD8B07D
:104E60000B1EC00E0FEC0DF0000EF86E640EF76E08
:104E7000260EF66E85EC0DF00BA053EF27F0C80E52
:104E80000FEC0DF0280E00EC0DF0CC0E0FEC0DF039
:104E9000290E00EC0DF0CF0E0FEC0DF0200E00EC03
:104EA0000DF065EF27F0C80E0FEC0DF0200E00ECB2
:104EB0000DF0CC0E0FEC0DF0280E00EC0DF0CF0E27
:104EC0000FEC0DF0290E00EC0DF082EC29F0D8B4B7
:104ED0000B6AFF0ED8B00B6E26EC25F083EC1EF0AB
:104EE000D8A03CEF27F0D8900BB0D88012000B6A06
:104EF000D8B00B1EC80E0FEC0DF0000EF86E640E4D
:104F0000F76E640EF66E85EC0DF00BA09CEF27F0AB
:104F1000C80E0FEC0DF0280E00EC0DF0CC0E0FECCF
:104F20000DF0290E00EC0DF0CF0E0FEC0DF0200E61
:104F300000EC0DF0AEEF27F0C80E0FEC0DF0200ED8
:104F400000EC0DF0CC0E0FEC0DF0280E00EC0DF087
:104F5000CF0E0FEC0DF0290E00EC0DF082EC29F0D5
:104F6000D8B40B6AFF0ED8B00B6E26EC25F083EC9C
:104F70001EF0D8A085EF27F0D8900BB0D880120093
:104F80000001BB65BB51B961B95112000001E8696C
:104F900000019D6FD0EF27F000019D6F0001E86BCD
:104FA000C80E9DEC0BF09DC0E8FF0001136E146A63
:104FB000156A166A15EC0EF00001E867EEEF27F0AF
:104FC000CD0E0FEC0DF0275000EC0DF0285000EC4A
:104FD0000DF0295000EC0DF0FDEF27F0CC0E0FEC9A
:104FE0000DF0275000EC0DF0285000EC0DF02E0EC7
:104FF00000EC0DF0295000EC0DF0A8EC29F00001B8
:10500000D8A409EF28F09D2BBB519D619D6F14EF33
:1050100028F0D8A014EF28F09D51B96114EF28F0C2
:105020009D07B9519D659D6F26EC25F083EC1EF020
:10503000D8A0D0EF27F000019D51120056EC25F0CA
:10504000FA0E9DEC0BF0E7CFE8FFE7BEE81EE7BEE7
:10505000E82A0001136E146A156A166A15EC0EF040
:10506000CB0E0FEC0DF0200EE7BE2D0E00EC0DF078
:10507000275000EC0DF0285000EC0DF0295000EC0A
:105080000DF0250E00EC0DF0A8EC29F00001D8A4DD
:105090004DEF28F0E72A51EF28F0D8A051EF28F083
:1050A000E70626EC25F083EC1EF0D8A01EEF28F0D2
:1050B0000001EF6B120000011150BB5D1250BC5992
:1050C000D8B068EF28F0BB51116EBC51126E1200BF
:1050D000B951115CBA511258D8B073EF28F0B951D8
:1050E000116EBA51126E12005BEC28F00001BE6B1B
:1050F0000001B851E812D8B486EF28F0B851E16E3B
:10510000000EE26E11C0E6FF12C0E7FF320E9DEC0A
:105110000BF011C013F012C014F0D89014321332F7
:10512000156A166A15EC0EF0C90E0FEC0DF026503C
:1051300000EC0DF02E0E00EC0DF0275000EC0DF001
:10514000285000EC0DF0295000EC0DF06D0E00EC35
:105150000DF0530E00EC0DF0A8EC29F00001D8A4DE
:10516000C1EF28F0112AD8B4122A112AD8B4122A71
:10517000BC51126274EF28F0BB511160116E74EFD4
:1051800028F0D8A0D3EF28F01106D8A012061106F7
:10519000D8A01206BA51126274EF28F0B951116406
:1051A000116E74EF28F0000133A2BE6933BCDEEF4C
:1051B00028F00001A00E116E0F0E126E000133BE1A
:1051C000E7EF28F00001D00E116E070E126E26ECEC
:1051D00025F083EC1EF0D8A078EF28F01200C00E66
:1051E0000FEC0DF00FC0F6FF10C0F7FF85EC0DF0CF
:1051F000FA0E9DEC0BF0A8EC29F0D8A406EF29F0EC
:10520000110E0F26D8B0102A0DEF29F0D8A01AEFF2
:1052100029F0130E0F26D8B0102A0FC0F6FF10C0C9
:10522000F7FFF86A0900F5CF0FF00900F5CF10F08D
:10523000EFEF28F026EC25F083EC1EF0D8A0EFEF7E
:1052400028F0150E0F26D8B0102A0FC0F6FF10C098
:10525000F7FFF86A0900F5CF0AF00900F550CEC053
:10526000E1FFCFC0E2FF0AC0E7FF12000F0BE8B674
:10527000080B0C0DF3CF13F0F4CF14F00001BE0EA9
:1052800013266F0E1422CC0E0FEC0DF013C0F6FF98
:1052900014C0F7FF85EC0DF0FA0E9DEC0BF0A8ECB6
:1052A00029F0D8A45AEF29F0050E1326D8B0142AF5
:1052B00061EF29F0D8A06EEF29F0070E1326D8B0C1
:1052C000142A13C0F6FF14C0F7FFF86A0900F5CFDF
:1052D00013F00900F5CF14F043EF29F026EC25F088
:1052E00083EC1EF0D8A043EF29F0090E1326D8B0A6
:1052F000142A13C0F6FF14C0F7FFF86A0900F5CFAF
:10530000E8FF1200040E93EC08F0040E93EC08F092
:10531000C5C0E8FFC35EC6C0E8FFC45AC4BE9BEF69
:1053200029F0640EC35E000EC45AC4BEA5EF29F076
:10533000D884D8901200640EC326000EC422C4AED6
:10534000A5EF29F0D894D8801200D894D8901200F4
:10535000050E93EC08F0050E93EC08F0C7C0E8FFCB
:10536000C35EC8C0E8FFC45AC4BEC1EF29F0640ED2
:10537000C35E000EC45AC4BECBEF29F0D884D890C7
:105380001200640EC326000EC422C4AECBEF29F077
:10539000D894D8801200D894D8901200C8EF2AF080
:1053A000800E0FEC0DF0000EF86E650EF76EEE0E2F
:1053B000F66E85EC0DF015EF2BF00101060E1E6F59
:1053C000660E1F6F0101F20E206F670E216F58EC01
:1053D0002AF0A9EC1EF000C2E8FF3AEC1FF067ECDF
:1053E0001FF0120001011E0E1E6F660E1F6F0101DD
:1053F000E40E206F680E216F58EC2AF0E9EF29F0D7
:105400000101360E1E6F660E1F6F0101CE0E206F5A
:105410006A0E216F58EC2AF0E9EF29F001014E0ED7
:105420001E6F660E1F6F01012A0E206F700E216F16
:1054300058EC2AF0E9EF29F00101660E1E6F660EA6
:105440001F6F0101F80E206F760E216F58EC2AF0C5
:10545000E9EF29F00001DD6B01017E0E1E6F660E83
:105460001F6F0101020E206F7D0E216F58EC2AF094
:10547000E9EF29F00101960E1E6F660E1F6F010104
:105480004A0E206F810E216F58EC2AF0E9EF29F0C7
:105490000101AE0E1E6F660E1F6F0101C40E206F5C
:1054A000840E216F58EC2AF0E9EF29F046EF31F035
:1054B0004FEC25F020C10DF021C10EF080EC25F05D
:1054C0000DC020F10EC021F1EAC026F1EBC027F19A
:1054D00000011150090AD8A4BAEF2AF00FC00DF04C
:1054E00010C00EF080EC25F00DC022F10EC023F1AB
:1054F000EAC028F1EBC029F100011150090AD8A433
:10550000A2EF2AF00FC00DF010C00EF080EC25F0D5
:105510000DC024F10EC025F1EAC02AF1EBC02BF139
:1055200057EC26F00001CDB1A8EF2AF02AC10FF008
:105530002BC110F04BEC26F024C10DF025C10EF06C
:1055400086EF2AF057EC26F00001CDB1BFEF2AF02C
:1055500028C10FF029C110F04BEC26F020C10DF04E
:1055600021C10EF064EC0DF022C10DF023C10EF04C
:1055700072EF2AF057EC26F00001CDB1120026C1DF
:105580000FF027C110F04BEC26F058EF2AF0120074
:1055900000C2E8FFBAEC1EF0800E0FEC0DF0000E1A
:1055A000F86E630EF76EF00EF66E85EC0DF08D0E54
:1055B0000FEC0DF0020100510001136E146A156A20
:1055C000166AE3EC0DF0CDEC05F0FA0E9DEC0BF055
:1055D000A8EC29F0D8A4F7EF2AF0610E0201002B05
:1055E0000063C8EF2AF0010E006FC8EF2AF0D8A0C0
:1055F00005EF2BF002010007000E0063C8EF2AF050
:10560000600E0201006FC8EF2AF083EC1EF0D8A0F4
:10561000E8EF2AF000C2E8FF0FEC1FF000C2E8FF3D
:10562000E8CFA5F0A9EC1EF01200C00E0FEC0DF0B3
:10563000CDEC05F0000EE16E030EE26E960E9DECD1
:105640000BF0C00EE1240FEC0DF0E75000EC0DF074
:10565000C00EE1240FEC0DF00E0E0FEC0DF082ECFD
:1056600029F0D8A43DEF2BF0E12A0F0EE1641EEFE4
:105670002BF0000EE16E1EEF2BF0D8A049EF2BF0BF
:10568000E106FF0EE1621EEF2BF00F0EE16E1EEF42
:105690002BF0A8EC29F0D8A454EF2BF0E72A7A0ECF
:1056A000E760E76E1EEF2BF0D8A05DEF2BF0E7066A
:1056B000200EE764E76E1EEF2BF083EC1EF0D8A0FF
:1056C0002FEF2BF00C0E0FEC0DF000C2E8FF3AECC0
:1056D0001FF012000DC02CF10EC02DF10FC02EF1E5
:1056E00010C02FF1D0C00DF0D1C00EF00001E80EB7
:1056F0000F6E030E106E67EC10F00001000E176EB7
:10570000010E186E6BEC11F013C0D0F014C0D1F084
:105710000001D251D027D351D123D4C00DF0D5C030
:105720000EF00001E80E0F6E030E106E67EC10F025
:105730000001000E176E010E186E6BEC11F0D2C056
:10574000D4F0D3C0D5F01350D45F1450D55B2CC126
:105750000DF02DC10EF02EC10FF02FC110F0120070
:105760000DC02CF10EC02DF10FC02EF110C02FF185
:10577000D0C00DF0D1C00EF0D2510D5ED3510E5AF3
:105780000001000E0F6E010E106E67EC10F00001AC
:10579000E80E176E030E186E6BEC11F013C0D0F00C
:1057A00014C0D1F0D2C00DF0D3C00EF0D4510D5EB4
:1057B000D5510E5A0001000E0F6E010E106E67ECEF
:1057C00010F00001E80E176E030E186E6BEC11F06E
:1057D00013C0D4F014C0D5F02CC10DF02DC10EF0C3
:1057E0002EC10FF02FC110F012000DC02CF10EC011
:1057F0002DF10FC02EF110C02FF10001BEA12DEF31
:105800002CF0000E00010F18D8B418EF2CF0D2C005
:1058100013F0D3C014F0D89013361436D051135E61
:10582000D151145A13C0D4F014C0D5F02DEF2CF080
:10583000000E00010F18D8B42DEF2CF0D2C013F0D9
:10584000D3C014F0D89013361436D451135ED5510A
:10585000145A13C0D0F014C0D1F02CC10DF02DC1DA
:105860000EF02EC10FF02FC110F012003C0E0001FF
:10587000B86F0001110EB56F030EB66F0001D00EA8
:10588000B36F000EB46F0B0EB76F57EC23F0DB6BEA
:105890006AEC2BF012003A0E0001B86F00011C0EEA
:1058A000B56F030EB66F3EEF2CF03E0E0001B86FE1
:1058B0000001270EB56F030EB66F3EEF2CF000010E
:1058C000110EB36F030EB46FF5EC2BF0DBA1D86BA8
:1058D000B0EC2BF00001D00EB56F000EB66F0B0EC2
:1058E000B76F57EC23F00001B86B120000011C0EDB
:1058F000B36F030EB46F64EF2CF00001270EB36F8B
:10590000030EB46F64EF2CF00DC02CF10EC02DF11E
:105910000FC02EF110C02FF1030132C30DF033C3BD
:105920000EF00001E80E0F6E030E106E67EC10F023
:105930000001000E176E010E186E6BEC11F013C013
:1059400032F314C033F3030134513227355133237A
:105950002CC10DF02DC10EF02EC10FF02FC110F093
:1059600012000DC02CF10EC02DF10FC02EF110C091
:105970002FF132C30DF033C30EF003013451000197
:105980000D5E0301355100010E5A0001000E0F6E2D
:10599000010E106E67EC10F00001E80E176E030E9A
:1059A000186E6BEC11F013C032F314C033F32CC13A
:1059B0000DF02DC10EF02EC10FF02FC110F000011F
:1059C000B86B1200420E0001B86F00013A0EB56FBD
:1059D000030EB66F0001D00EB36F000EB46F040E4D
:1059E000B76F57EC23F06AEC2BF01200440E000165
:1059F000B86F00013E0EB56F030EB66FEAEF2CF0E4
:105A0000460E0001B86F0001420EB56F030EB66F6F
:105A1000EAEF2CF000013A0EB36F030EB46FB0EC56
:105A20002BF00001D00EB56F000EB66F040EB76FED
:105A300057EC23F00001B86B120000013E0EB36F6B
:105A4000030EB46F0FEF2DF00001420EB36F030E83
:105A5000B46F0FEF2DF00001460EB56F030EB66F59
:105A60000001D00EB36F000EB46F060EB76F57EC87
:105A700023F06AEC2BF01200B0EC2BF00001D00EFA
:105A8000B56F000EB66F0001460EB36F030EB46F14
:105A9000060EB76F57EC23F00001B86B1200AEC2D0
:105AA000B9F0AFC2BAF0B0C2BBF0B1C2BCF01200E4
:105AB000CEC0B5F0CFC0B6F00001DC0EB36F000E63
:105AC000B46F050EB76F57EC23F0CEC0B3F0CFC064
:105AD000B4F00001DC51E83A0F0BE46FE36BDDBF7B
:105AE000E31FE16BDF51DDBDE16FE26BE051DDBB38
:105AF000E26F0F0EE117E217DD17DC17120000014D
:105B0000E451E83AF00BDC13E3BFDD8FE151E8121A
:105B1000D8B48EEF2DF0E151DF6FDD8DE251E81248
:105B2000D8B496EF2DF0E251E06FDD8B0001DC0E72
:105B3000B56F000EB66F050EB76F57EC23F012006D
:105B400010C4DFF011C4E0F01200DFC010F4E0C0B8
:105B500011F4120012C4DFF013C4E0F01200DFC031
:105B600012F4E0C013F4120014C4DFF015C4E0F026
:105B70001200DFC014F4E0C015F412000001DBAF26
:105B800012000301196B246B2F6B12000001DBAFB5
:105B90001200A7C313F0A8C314F083511326845135
:105BA000142213C0A7F314C0A8F3A9C313F0AAC307
:105BB00014F0855113268651142213C0A9F314C082
:105BC000AAF3ABC313F0ACC314F08751132688516A
:105BD000142213C0ABF314C0ACF312000001DBAF0E
:105BE00012000301A76BA86BA96BAA6BAB6BAC6B24
:105BF00012000001B96BB92B600E0001BB6F1200DF
:105C00000001DD51DD6706EF2EF01200020100C237
:105C10000AF0006F00010AC0DDF03AEC1FF000014D
:105C2000DDC00AF002010AC000F212000001DBAF81
:105C3000120003011951196B18C30AF000010D6E0F
:105C40000E6AE8BE0E680D360E360001640E0F6E49
:105C5000000E106E67EC10F00AC017F0186A6BECBB
:105C600011F013500301A727000114500301A823CA
:105C700003012451246B23C30AF000010D6E0E6A48
:105C8000E8BE0E680D360E360001640E0F6E000E73
:105C9000106E67EC10F00AC017F0186A6BEC11F088
:105CA00013500301A927000114500301AA23030183
:105CB0002F512F6B2EC30AF000010D6E0E6AE8BE45
:105CC0000E680D360E360001640E0F6E000E106E5B
:105CD00067EC10F00AC017F0186A6BEC11F0135063
:105CE0000301AB27000114500301AC231200000193
:105CF000DBAF1200A7EC31F0120057EC23F01200DA
:105D00000001D00EB36F000EB46FCEC0B5F0CFC09F
:105D1000B6F00B0EB76F57EC23F00001D00EB56F45
:105D2000000EB66FCEC0B3F0CFC0B4F00B0EB76F9D
:105D300012000201D890A23712000201D890A233BB
:105D400012000001E9AF120011EC10F0120013C2B2
:105D50000FF014C210F0030E0001A06F56EC30F0EB
:105D60000FC013F210C014F21200A9C20FF0AAC2A1
:105D700010F00D0E0001A06F56EC30F00FC0A9F22C
:105D800010C0AAF212000001DBAF12000501006B87
:105D9000016B1200C9EC0BF012000001CE51B36F81
:105DA000020EB46FCF5100011F6E030E7EEC08F09F
:105DB00014C08BF015C08CF0C00E0FEC0DF0000E6F
:105DC000F86E8A0EF76EDC0EF66E85EC0DF083EC45
:105DD0001EF0D8A0E7EF2EF000011F507EEC08F077
:105DE00014C06DF015C06EF014C06FF015C070F0E7
:105DF000FA0E9DEC0BF0C00E0FEC0DF0000EF86EDD
:105E00008A0EF76EEE0EF66E85EC0DF083EC1EF04A
:105E1000D8A006EF2FF000011F507EEC08F014C050
:105E20006BF015C06CF0FA0E9DEC0BF000016B519D
:105E30006D276C516E236E336D336E9F6FC017F0FC
:105E400070C018F00001E80E146E030E156E136A90
:105E5000166A6B51175E6C51185A18321732189E19
:105E6000196A1A6A6BEC11F013C06BF014C06CF075
:105E700000016B0EB56F000EB66F040E0001B76F18
:105E800057EC23F012000001CE51B36F020EB46F35
:105E9000CF5100011F6EC00E0FEC0DF0000EF86E1A
:105EA0008A0EF76EDC0EF66E85EC0DF083EC1EF0BC
:105EB000D8A056EF2FF000011F507EEC08F014C060
:105EC0006BF015C06CF0FA0E9DEC0BF0C00E0FECF1
:105ED0000DF0000EF86E8A0EF76EEE0EF66E85EC83
:105EE0000DF083EC1EF0D8A071EF2FF000011F50D1
:105EF0007EEC08F014C06DF015C06EF0FA0E9DEC4B
:105F00000BF00001E80E146E030E156E136A166A8C
:105F10006BC017F06CC018F0196A1A6A00016D5155
:105F2000175E6E51185A18AE97EF2FF0FF0E196ECC
:105F30001A6E6BEC11F013C06BF014C06CF0000122
:105F40006B0EB56F000EB66F040E0001B76F57EC05
:105F500023F012000001CE51B36F020EB46FCF5187
:105F600000011F6EC00E0FEC0DF0000EF86E8A0ED1
:105F7000F76ECA0EF66E85EC0DF083EC1EF0D8A01D
:105F8000BDEF2FF000011F507EEC08F0000113362A
:105F90001436153614C06DF015C06EF0FA0E9DEC77
:105FA0000BF0C00E0FEC0DF0000EF86E8A0EF76EBF
:105FB000DC0EF66E85EC0DF083EC1EF0D8A0DCEF65
:105FC0002FF000011F507EEC08F00001133614364C
:105FD000153614C06BF015C06CF0FA0E9DEC0BF08A
:105FE000C00E0FEC0DF0000EF86E8A0EF76EEE0E7E
:105FF000F66E85EC0DF083EC1EF0D8A0FBEF2FF0D1
:1060000000011F507EEC08F00001133614361536DF
:1060100014C06FF015C070F0FA0E9DEC0BF000018B
:10602000E80E146E030E156E136A166A6BC017F035
:106030006CC018F0196A1A6A00016D51175E6E5132
:10604000185A18AE25EF30F0FF0E196E1A6E6BEC71
:1060500011F013C06BF014C06CF00001E80E146E68
:10606000030E156E136A166A6DC017F06EC018F035
:10607000196A1A6A00016F51175E7051185A18AEEA
:1060800043EF30F0FF0E196E1A6E6BEC11F013C077
:106090006FF014C070F000016B0EB56F000EB66F9C
:1060A000060E0001B76F57EC23F01200140E9DECA2
:1060B0000BF00001A05193EC08F0C00E0FEC0DF0B6
:1060C000000EF86E670EF76E860EF66E85EC0DF01C
:1060D000CB0E0FEC0DF069C00DF06AC00EF067EC4E
:1060E00010F01450136E1550146E156A15EC0EF066
:1060F000200E0A6E300E25640AC025F0255000ECF3
:106100000DF0265000EC0DF02E0E00EC0DF0275097
:1061100000EC0DF0285000EC0DF0A8EC29F0D8A40C
:1061200098EF30F000010F2AD8B4102A56EF30F063
:10613000D8A0A2EF30F000010F06FF0E0F6010068E
:1061400056EF30F083EC1EF0D8A056EF30F012007E
:106150000201FF0EA563BAEF30F000019D510FEC74
:106160000DF0000EF86E640EF76E140EF66E85ECF0
:106170000DF012000201D1B1D8EF30F0D1A3D8EF69
:1061800030F000019D510FEC0DF0000EF86E640E22
:10619000F76E020EF66E85EC0DF000019D51080FB2
:1061A0000FEC0DF00201310EA52500EC0DF01200F0
:1061B0000201D1A10DEF31F0D1B30DEF31F00001AB
:1061C0009D510FEC0DF0000EF86E640EF76E6E0E22
:1061D000F66E85EC0DF000019D510E0F0FEC0DF0E9
:1061E0000201300EA52500EC0DF00201A551D8905A
:1061F000E836500F0001136E146A156A166A15EC22
:106200000EF000019D51040F0FEC0DF0285000EC32
:106210000DF0295000EC0DF012000201D1A1120086
:10622000D1A3120000019D510FEC0DF0000EF86E8D
:10623000640EF76EDA0EF66E85EC0DF000019D51DE
:106240000D0F0FEC0DF00201A55101010E2500010B
:10625000136E146A156A166AE3EC0DF00201A5517B
:10626000D890E836010F0001136E146A156A166A99
:1062700015EC0EF000019D51040F0FEC0DF02850AD
:1062800000EC0DF0295000EC0DF012000301FF0EA0
:10629000AD635BEF31F0C00E0FEC0DF0000EF86E49
:1062A000640EF76E140EF66E85EC0DF0FA0E9DEC92
:1062B0000BF067EF31F00301AD510201A56FC00E85
:1062C00000019D6FA8EC30F0FA0E9DEC0BF0A8ECED
:1062D00029F0D8A477EF31F0010110510301AD2B63
:1062E000AD6346EF31F0FF0EAD6F46EF31F0D8A051
:1062F00087EF31F00301AD07FE0EAD6346EF31F0DD
:1063000001011051E8060301AD6F46EF31F083EC57
:106310001EF0D8A067EF31F000C2E8FF3AEC1FF0A2
:106320001200000EF86E8B0EF76E000EF66E000E69
:106330000A6E020EE26E000EE16E0900F550E66E86
:106340000A060900F550E66E0A2E9DEF31F0000EA8
:10635000F86E8C0EF76E000EF66E000E0A6E030ECF
:10636000E26E000EE16E0900F550E66E0A060900C5
:10637000F550E66E0A2EB3EF31F0000EF86E8D0E7A
:10638000F76E000EF66E000E0A6E040EE26E000E40
:10639000E16E0900F550E66E0A060900F550E66E5A
:1063A0000A2EC9EF31F012002020202020202020CA
:1063B00020202020202020200000204D6963726FC3
:1063C0005374617220323030302000002020566536
:1063D0007273696F6E20322E3064202000004144B9
:1063E00043204348205858203D2058585858000012
:1063F000202020416972637261667420232020206E
:106400000000202020202035332E58204D487A20AF
:1064100020200000202020202020204F4646202041
:10642000202020200000204163636570743F2059C4
:106430006573204E6F20000020507265737320201A
:10644000204F7074696F6E200000202020202020D3
:1064500020002020202053747564656E7420202055
:106460002020000020596573204E6F200000203549
:10647000302E5858204D487A20204348582000009C
:1064800078426C642052504D203D2078787878789E
:1064900000005265747261637473206172652055E7
:1064A000502100002020466F726D617420466C619F
:1064B0007368202000002020466F726D6174696E41
:1064C000672E2E2E20200000202020436F70796937
:1064D0006E672E2E2E20202000002037322E585896
:1064E000204D487A20434858582000005245432008
:1064F000566F6C74733D2058582E585800005468DD
:10650000726F74746C65202041646A757374000046
:10651000202041494C20442F522048494748202000
:106520000000202041494C20442F5220204C4F573E
:10653000202000002020454C4520442F522048496F
:106540004748202000002020454C4520442F522061
:10655000204C4F5720200000202052554420442F2B
:10656000522048494748202000002020525544200E
:10657000442F5220204C4F57202000002020205331
:106580004E415020524947485420202000002020EE
:1065900020534E415020204C4546542020200000DE
:1065A0002020204155544F20205452494D20202076
:1065B0000000202020202050524553455420202008
:1065C0002020000020202043414C494252415445A4
:1065D00020202020000053656C65637420204169F1
:1065E00072637261667400EE65DE66000000204131
:1065F0006972637261667420206E616D65200006A9
:1066000066D66504000020202020202054696D6596
:10661000722020202020001E66EE65080000202049
:1066200020202020536E6170202020202020003662
:106630006606660C00002020202020536572766FCD
:10664000732020202020004E661E661000002020AF
:106650002020204D6978657273202020202000665C
:10666000663666140000202020202053776974636A
:10667000682020202020007E664E66180000202022
:1066800020204F7074696F6E7320202020200096A8
:106690006666661C000020536861726564204F7056
:1066A00074696F6E732000AE667E66200000202045
:1066B00053797374656D205365747570202000C61E
:1066C00066966624000053656C65637420467265A7
:1066D0007175656E637900DE66AE66280000202065
:1066E000202020204558495420202020202000D65A
:1066F00065C6662C0000456E61626C652020202016
:1067000020202020202000005265736574203F2047
:10671000202020202020202000005A65726F202099
:106720003F2020202020202020200000436C656195
:1067300072203F20202020202020202000004169BE
:1067400072637261667420232020202020200000C4
:10675000546F204146542023202020202020202038
:106760000000426C61646573203D202020202020C1
:106770002020000046786420467273742020202078
:10678000202020200000566F6C74732020202020D1
:1067900020202020202000005769647468202020D9
:1067A000202020202020202000004368616E6E659C
:1067B0006C73202020202020202000004E6567538D
:1067C000686966743F202020202020200000506F40
:1067D00073203D2020202020202020202020000089
:1067E0004761696E202020202020202020202020AA
:1067F00000002020202020204D6F646520202020D4
:106800002020000E68826800809C68BD03004D69EE
:106810006E75746573202020202020202020002EFB
:1068200068F2670540BF0300000000FF00005365E9
:10683000636F6E6473202020202020202020004ED3
:10684000680E680540BE0300000000FF0000204500
:106850006E61626C652020537769746368200068FC
:10686000682E680680C003005468726F74746C658B
:1068700020202020202020200082684E680100C1B6
:10688000030045584954202020202020202020208B
:10689000202000F26768680300CD0000202020203F
:1068A00055502054696D65722020202000B468CCBA
:1068B00068000000202020446F776E2054696D65C9
:1068C0007220202000CC689C68010000446F776E25
:1068D000202053746F702054696D6572009C68B4F9
:1068E0006802000053522041494C202020202020E3
:1068F00020202020000469B46A01404C030000FFFE
:10690000007E0000535220454C45202020202020AE
:1069100020202020002469E46801404E030000FF8D
:10692000007E000053522052554420202020202079
:10693000202020200044690469014050030000FF2A
:10694000007E000053522054485420202020202054
:10695000202020200064692469014052030000FFC8
:10696000007E000053522041494C203F202020202F
:1069700020202020007E69446903004D030053520B
:1069800020454C45203F202020202020202000981A
:1069900069646903004F0300535220525544203F5D
:1069A000202020202020202000B2697E6903005191
:1069B0000300535220544854203F20202020202000
:1069C000202000CC6998690300530300534C2041F8
:1069D000494C2020202020202020202000EC69B2DB
:1069E00069014054030000FF007E0000534C204525
:1069F0004C4520202020202020202020000C6ACC84
:106A000069014056030000FF007E0000534C2052F5
:106A1000554420202020202020202020002C6AEC1B
:106A200069014058030000FF007E0000534C2054D1
:106A3000485420202020202020202020004C6A0CB8
:106A40006A01405A030000FF007E0000534C2041C1
:106A5000494C203F202020202020202000666A2C46
:106A60006A0300550300534C20454C45203F20202D
:106A700020202020202000806A4C6A030057030059
:106A8000534C20525544203F2020202020202020FD
:106A9000009A6A666A0300590300534C2054485414
:106AA000203F202020202020202000B46A806A037C
:106AB000005B03004558495420202020202020203E
:106AC0002020202000E4689A6A0300CD00002020E6
:106AD000202041696C65726F6E202020202000EE1E
:106AE0006AE86B0986026C0000BE586C58002020D2
:106AF0002020456C657661746F7220202020000E86
:106B00006BCE6A0986026C0000EC58965800202073
:106B10002020205275646465722020202020002EE1
:106B20006BEE6A0986026C0000FA58AA5800202011
:106B300020205468726F74746C6520202020004EF1
:106B40006B0E6B0986F86C00006259085900202012
:106B50002020202043483520202020202020006EA7
:106B60006B2E6B0986EA6D0000145AC45900202070
:106B70002020202043483620202020202020008E66
:106B80006B4E6B0986EA6D00003A5AEC59002020E2
:106B9000202020204348372020202020202000AE25
:106BA0006B6E6B0986EA6D0000485A005A0020207F
:106BB000202020204348382020202020202000CEE4
:106BC0006B8E6B0986406E0000785A565A00202062
:106BD0002020537562205472696D7320202000E8D4
:106BE0006BAE6B0980B46E004558495420202020BC
:106BF000202020202020202000CE6ACE6B0300CD54
:106C0000000052542F44574E2020202020202020C6
:106C1000202000206CDE6C0202D00000009E5A0092
:106C200043656E74657220202020202020202020C3
:106C3000003E6C026C0202D20000009E5A004C54CE
:106C40002F55502020202020202020202020005CB4
:106C50006C206C0202D40000009E5A004475616CE6
:106C600020526174652020202020202000766C3E78
:106C70006C0100D600005472696D20202020202075
:106C800020202020202000906C5C6C0100D70000A8
:106C90004154205253542020202020202020202006
:106CA00000AA6C766C0300DB00004578706F20480A
:106CB0004920202020202020202000C46C906C013E
:106CC00000D900004578706F204C4F5720202020BD
:106CD0002020202000DE6CAA6C0100DA000045585C
:106CE0004954202020202020202020202020000285
:106CF0006CC46C0300CD0000486967682020202028
:106D0000202020202020202000166D886D020332D4
:106D10000340009E5A004C6F772020202020202026
:106D200020202020202000346DF86C020334034022
:106D3000009E5A005472696D2020202020202020BF
:106D400020202020004E6D166D0100360300547285
:106D5000696D204D6F646520202020202020006A6E
:106D60006D346D0000A26D37030050726573657459
:106D70002020202020202020202000886D4E6D0221
:106D800003380340009E5A004558495420202020D3
:106D9000202020202020202000F86C6A6D0300CDE8
:106DA00000005472696D204D6F6465204E4F524D46
:106DB000414C00BA6DD26D0000005472696D204DD7
:106DC0006F6465202020204C4F5700D26DA26D01CA
:106DD00000005472696D204D6F6465202020484981
:106DE000474800A26DBA6D020000486967682F55D8
:106DF0007020202020202020202000086E266E02F7
:106E000002D00000009E5A004C6F772F44574E204E
:106E1000202020202020202000266EEA6D0202D2B1
:106E20000000009E5A004558495420202020202070
:106E300020202020202000EA6D086E0300CD0000F5
:106E40004120202020202020202020202020202021
:106E5000005E6E9A6E0203D00048009E5A004220E7
:106E60002020202020202020202020202020007CE6
:106E70006E406E0203D20048009E5A00432020203C
:106E8000202020202020202020202020009A6E5E1C
:106E90006E0203D40048009E5A00455849542020F1
:106EA0002020202020202020202000406E7C6E0307
:106EB00000CD000041696C65726F6E20202020209B
:106EC0002020202000D26EA46F010208040000FAE6
:106ED0004A00456C657661746F7220202020202066
:106EE000202000F06EB46E010209040000FA4A008E
:106EF00052756464657220202020202020202020EC
:106F0000000E6FD26E01020A040000FA4A005468B3
:106F1000726F74746C652020202020202020002CAB
:106F20006FF06E01020B040000FA4A00434835205E
:106F3000202020202020202020202020004A6F0E0A
:106F40006F01020C040000FA4A004348362020205A
:106F50002020202020202020202000686F2C6F017E
:106F6000020D040000FA4A00434837202020202068
:106F7000202020202020202000866F4A6F01020E52
:106F8000040000FA4A004348382020202020202016
:106F900020202020202000A46F686F01020F040031
:106FA00000FA4A0045786974202020202020202003
:106FB0002020202000B46E866F0300CD00004E6FAD
:106FC0006E6500CA6F1E700000002041494C00D65B
:106FD0006FBE6F01000020454C4500E26FCA6F0292
:106FE00000002052554400EE6FD66F03000020547D
:106FF000485400FA6FE26F04000020434835000651
:1070000070EE6F05000020434836001270FA6F06DC
:10701000000020434837001E700670070000204320
:10702000483800BE6F1270080000202020204D4913
:1070300058455220314120202020004A70E2720938
:10704000864A735C03FE5AB05A00202020204D4926
:1070500058455220314220202020006A702A7009B1
:10706000864A736103FE5AB05A00202020204D4901
:1070700058455220314320202020008A704A700950
:10708000864A736603FE5AB05A00202020204D49DC
:107090005845522031442020202000AA706A7009EF
:1070A000864A736B03FE5AB05A00202020204D49B7
:1070B0005845522032412020202000CA708A700991
:1070C000864A737003FE5AB05A00202020204D4992
:1070D0005845522032422020202000EA70AA700930
:1070E000864A737503FE5AB05A00202020204D496D
:1070F00058455220324320202020000A71CA7009CE
:10710000864A737A03FE5AB05A00202020204D4947
:1071100058455220324420202020002A71EA70096C
:10712000864A737F03FE5AB05A00202020204D4922
:1071300058455220334120202020004A710A71090D
:10714000864A738403FE5AB05A00202020204D49FD
:1071500058455220334220202020006A712A7109AC
:10716000864A738903FE5AB05A00202020204D49D8
:1071700058455220334320202020008A714A71094B
:10718000864A738E03FE5AB05A00202020204D49B3
:107190005845522033442020202000AA716A7109EA
:1071A000864A739303FE5AB05A0020202041494C6E
:1071B00020746F2052554420202000CA718A710922
:1071C00086FC7293034A5B405B00202020525544AA
:1071D00020746F2041494C20202000EA71AA7109D7
:1071E00086FC7293035E5B545B0020202052554462
:1071F00020746F20454C45202020000A72CA710976
:1072000086FC729303725B685B0020202054485414
:1072100020746F20454C45202020002672EA710121
:10722000881604E067002020202020565441494C55
:107230002020202020200042720A7203889803F642
:1072400066002020202020454C45564F4E2020200F
:107250002020005E72267203889903F666002020C3
:1072600020204455414C2041494C202020200078CA
:107270007242720980507400202020204455414CF5
:1072800020454C45202020200092725E720980EC3F
:1072900074002020202054485420484F4C44202083
:1072A000202000AC72787209803A750020202020DE
:1072B00049444C45202055502020202000C6729281
:1072C00072098088750020204D6978657220206FD2
:1072D00072646572202000E272AC720388A40374A9
:1072E00067004558495420202020202020202020BD
:1072F0002020002A70C6720300CD0000506F73205A
:107300006761696E20202020202020200016733025
:10731000730100DF00004E6567206761696E202001
:10732000202020202020003073FC720100E00000AB
:107330004558495420202020202020202020202093
:1073400000FC7216730300CD000046726F6D2020A2
:107350002020202020202020202000647336740468
:1073600000DC00005461626C652020202020202079
:10737000202020200080734A730000F075E4000094
:10738000546F20202020202020202020202020207A
:10739000009A7364730400DD00005265706C6163D1
:1073A0006520202020202020202000B4738073033B
:1073B00000E300005A502020202020202020202000
:1073C0002020202000CE739A730100DE0000506F51
:1073D00073206761696E202020202020202000E893
:1073E00073B4730100DF0000506F7320496E642096
:1073F0002020202020202020000274CE730400E1F1
:1074000000004E6567206761696E202020202020E3
:107410002020001C74E8730100E000004E65672026
:10742000496E642020202020202020200036740275
:10743000740400E2000045584954202020202020F8
:10744000202020202020004A731C740300CD00005F
:10745000456E61626C6520202020202020202020A5
:10746000006A74D27403009A030052657620434880
:1074700037202020202020202020008474507403F6
:10748000009B030044494646202020202020202045
:1074900020202020009E746A7401009C0300466C2A
:1074A000617020202020202020202020202000B8D3
:1074B00074847401009D030043524F572020202004
:1074C000202020202020202000D2749E740300C69B
:1074D000030045584954202020202020202020202F
:1074E0002020005074B8740300CD0000456E616226
:1074F0006C652020202020202020202000067520E0
:10750000750300170400526576204348362020207A
:10751000202020202020002075EC74030018040097
:1075200045584954202020202020202020202020A1
:1075300000EC7406750300CD0000456E61626C6559
:10754000202020202020202020200054756E75034C
:10755000009E0300506F736974696F6E20202020B5
:1075600020202020006E753A7501009F03004558C9
:107570004954202020202020202020202020003AB4
:107580007554750300CD0000456E61626C65202066
:10759000202020202020202000A275D6750300A0E6
:1075A0000300506F736974696F6E204120202020A2
:1075B000202000BC7588750100A10300506F73691D
:1075C00074696F6E204220202020202000D675A2F2
:1075D000750100A203004558495420202020202096
:1075E000202020202020008875BC750300CD0000DD
:1075F0005461626C65202020202020204E6F6E6533
:10760000000876E07600000041697263726166747A
:10761000205461626C652031002076F0750900000D
:107620004169726372616674205461626C652032D4
:1076300000387608760A0000476C6F6162616C2042
:107640005461626C65202031005076207601000084
:10765000476C6F6162616C205461626C65202032FE
:107660000068763876020000476C6F6162616C20BA
:107670005461626C652020330080765076030000F0
:10768000476C6F6162616C205461626C65202034CC
:107690000098766876040000476C6F6162616C2028
:1076A0005461626C6520203500B07680760500005C
:1076B000476C6F6162616C205461626C652020369A
:1076C00000C8769876060000476C6F6162616C2096
:1076D0005461626C6520203700E076B076070000C8
:1076E000476C6F6162616C205461626C6520203868
:1076F00000F075C876080000202020202041494C69
:107700002044522020202020001277E6780680AE08
:1077100003002020202020454C45204452202020DA
:107720002020002C77F8760680AF03002020202050
:107730002052554420445220202020200046771219
:10774000770680B00300202020202050524553456A
:107750005420202020200060772C770680B1030081
:10776000202020204D495845522020312020202023
:10777000007A7746770680B20300202020204D490A
:107780005845522020322020202000947760770630
:1077900080B30300202020204D495845522020333B
:1077A0002020202000AE777A770680B403002020C6
:1077B000202020204348352020202020202000C8E1
:1077C0007794770680B50300202020204155544F40
:1077D000205452494D20202000E277AE770680B633
:1077E0000300202020202043483820412020202052
:1077F000202000FC77C8770680B7030020202020D7
:10780000204348382042202020202020001678E203
:10781000770680B8030020202020204348382043EA
:10782000202020202020003078FC770680B903003B
:1078300020202020534E4150202052202020202064
:10784000004A7816780680BB030020202020534E83
:10785000415020204C2020202020006478307806E1
:1078600080BC0300205468726F74746C65202048DB
:107870006F6C6420007E784A780680C20300202066
:107880002049646C6520557020203120202000980C
:107890007864780680C3030020202049646C65204A
:1078A000557020203220202000B2787E780680C4D7
:1078B000030020202020202043524F57202020204A
:1078C000202000CC7898780680C503002054726987
:1078D0006767657220506F696E74732000E678B236
:1078E0007809800079004558495420202020202024
:1078F00020202020202000F876CC780300CD000046
:1079000041696C65726F6E205472696720506F73A5
:10791000001C7970790188C903CE6700456C6576D3
:1079200061746F722054726720506F730038790051
:10793000790188CA03CE670052756464657220209D
:107940005472696720506F730054791C790188CB99
:1079500003CE67005468726F74746C65205472674C
:1079600020506F7300707938790188CC03CE67009E
:10797000455849542020202020202020202020204D
:1079800000007954790300CD000020202020202021
:10799000204F4E2020202020202000A279EA7C10B9
:1079A0000000202020202020204F4646202020209C
:1079B000202000BA798A79200000535741202020E6
:1079C00020202020202020204F4E00D279A27900B4
:1079D0000000535741202020202020202020204F2D
:1079E000464600EA79BA79800000535742202020A9
:1079F00020202020202020204F4E00027AD2790122
:107A00000000535742202020202020202020204FFB
:107A10004646001A7AEA7981000053574320202015
:107A200020202020202020204F4E00327A027A028F
:107A30000000535743202020202020202020204FCA
:107A40004646004A7A1A7A82000053574420202082
:107A50002020202020505245535300627A327A83EE
:107A6000000053574420202020202052454C4541FF
:107A70005345007A7A4A7A03000053574520202064
:107A800020202020202020204F4E00927A627A046D
:107A90000000535745202020202020202020204F68
:107AA000464600AA7A7A7A8400005357462020205E
:107AB00020202020202020204F4E00C27A927A05DC
:107AC0000000535746202020202020202020204F37
:107AD000464600DA7AAA7A850000535747202020CC
:107AE00020202020202020204F4E00F27AC27A064B
:107AF0000000535747202020202020202020204F06
:107B00004646000A7BDA7A86000053574820202038
:107B100020202020202020204F4E00227BF27A07B8
:107B20000000535748202020202020202020204FD4
:107B30004646003A7B0A7B870000535749202020A5
:107B40002020202020505245535300527B227B8915
:107B5000000053574920202020202052454C454109
:107B60005345006A7B3A7B09000053574A20202086
:107B70002020202020202020204100827B527B8B4F
:107B8000000053574A2020202020202020202020A1
:107B90002042009A7B6A7B4B000053574A202020EA
:107BA0002020202020202020204300B27B827B8CBC
:107BB000000053574B202020202020202020202070
:107BC0004F4E00CA7B9A7B0D000053574B2020205C
:107BD000202020202020204F464600E27BB27B8DD3
:107BE000000053574C2020202020202020505245B8
:107BF000535300FA7BCA7B8E000053574C20202041
:107C000020202052454C4541534500127CE27B0E1A
:107C1000000053574D202020202020202050524586
:107C20005353002A7CFA7B8F000053574D202020AD
:107C300020202052454C4541534500427C127C0F88
:107C4000000041696C65726F6E202020202020208A
:107C50004F4E005A7C2A7C30000041696C65726F7F
:107C60006E2020202020204F464600727C427CB0AF
:107C70000000456C657661746F7220202020202002
:107C80004F4E008A7C5A7C310000456C65766174E9
:107C90006F7220202020204F464600A27C727CB1CB
:107CA000000052756464657220202020202020206E
:107CB0004F4E00BA7C8A7C32000052756464657253
:107CC000202020202020204F464600D27CA27CB2DB
:107CD00000005468726F74746C652020202020208E
:107CE0004F4E00EA7CBA7C3300005468726F7474A3
:107CF0006C6520202020204F4646008A79D27CB334
:107D000000002020204175746F20205472696D207E
:107D10002020001C7D267E0980B67F005265736599
:107D200074204175746F205472696D73003A7D023E
:107D30007D038CDB0008677C5B0020202054726987
:107D40006D20205A65726F20202000587D1C7D0315
:107D50008CDB001A678C5B00436C65617220547287
:107D6000696D205A65726F7300767D3A7D038CDBF6
:107D7000002C67DC5B0020416C742020204169727C
:107D800063726166742000907D587D0980407E009A
:107D900020436F707920204169726372616674209C
:107DA00000B07D767D058EDD005067005CF25B00E3
:107DB00020205365742044656661756C74732020BF
:107DC00000CE7D907D038CDB000867EE5C004E7575
:107DD0006D202070726F7020626C6164657300EEBC
:107DE0007DB07D05C8A503626701000500005265EE
:107DF000747261637473205761726E696E67000AF2
:107E00007ECE7D0388A603F66600204155584F5567
:107E10005420436F6E74726F6C2000267EEE7D00DE
:107E2000807280BA0200455849542020202020202A
:107E300020202020202000027D0A7E0300CD0000AB
:107E400020416C742023312020202020202020205D
:107E500000607E9C7F0540CF0300000000600000B2
:107E600020416C742020233120537769746368208B
:107E7000007A7E407E0680CE030020416C74202371
:107E800032202020202020202020009A7E607E05A5
:107E900040D1030000000060000020416C742020ED
:107EA0002332205377697463682000B47E7A7E069B
:107EB00080D0030020416C74202333202020202018
:107EC0002020202000D47E9A7E0540D303000000AD
:107ED0000060000020416C74202023332053776918
:107EE0007463682000EE7EB47E0680D203002041D9
:107EF0006C74202334202020202020202020000EFD
:107F00007FD47E0540D503000000006000002041C2
:107F10006C74202023342053776974636820002810
:107F20007FEE7E0680D4030020416C742023352030
:107F3000202020202020202000487F0E7F0540D7D1
:107F4000030000000060000020416C7420202335F5
:107F5000205377697463682000627F287F0680D68B
:107F6000030020416C742023362020202020202074
:107F7000202000827F487F0540D903000000006078
:107F8000000020416C7420202336205377697463ED
:107F90006820009C7F627F0680D8030045584954C2
:107FA00020202020202020202020202000407E8211
:107FB0007F0300CD00004154206D6F6465202020B8
:107FC00020202020202000D27F248000003E80B688
:107FD000020041542073746570202020202020204E
:107FE000202000EC7FB67F05009E020041542074E3
:107FF00069636B732020202020202020000680D27F
:108000007F05009F0200746F20545A2020202020FA
:10801000202020202020002480EC7F0304DB0000AF
:10802000002C5C004558495420202020202020208E
:108030002020202000B67F06800300CD00004154A0
:10804000206D6F6465202020202020496E63005839
:108050008058800000B602004154206D6F64652096
:108060004F6E652053686F74003E803E800100B6FD
:1080700002002020202020202043483120202020E2
:108080002020008A80328101000020202020202032
:108090002043483220202020202000A2807280032C
:1080A00000002020202020202043483320202020B2
:1080B000202000BA808A8005000020202020202077
:1080C0002043483420202020202000D280A2800796
:1080D0000000202020202020204348352020202080
:1080E000202000EA80BA80090000202020202020E3
:1080F00020434836202020202020000281D2800BFF
:10810000000020202020202020434837202020204D
:108110002020001A81EA800D00002020202020204D
:108120002043483820202020202000328102810F67
:1081300000002020202020202050504D20202020F2
:1081400020200072801A8180000020202042756467
:1081500064792020426F782020200064817E81098C
:108160008098810020202020205461626C6573205B
:1081700020202020007E814A8109803282004558DB
:108180004954202020202020202020202020004A88
:108190008164810300CD00004D6173746572203FDE
:1081A000202020202020202000B281E8810300A18F
:1081B000020020204D617374657220204D6F64654C
:1081C000202000CE81988100000282B70200537403
:1081D0007564656E74203F2020202020202000E858
:1081E00081B2810300A0020045584954202020207C
:1081F0002020202020202020009881CE810300CD47
:1082000000004D204D6F64653D4D6963726F53747E
:108210006172001A821A820000004D204D6F646561
:108220003D46757461626120202000028202820155
:1082300000004169726372616674205461626C650A
:108240002031005282728309868C83DA03FA5C0043
:108250005D004169726372616674205461626C658D
:108260002032007282328209868C83E503FA5C0038
:108270005D00476C6F62616C20205461626C652008
:108280002031009282528209868C834602FA5C0079
:108290005D00476C6F62616C20205461626C6520E8
:1082A000203200B282728209868C835102FA5C000D
:1082B0005D00476C6F62616C20205461626C6520C8
:1082C000203300D282928209868C835C02FA5C00A1
:1082D0005D00476C6F62616C20205461626C6520A8
:1082E000203400F282B28209868C836702FA5C0035
:1082F0005D00476C6F62616C20205461626C652088
:108300002035001283D28209868C837202FA5C00C7
:108310005D00476C6F62616C20205461626C652067
:108320002036003283F28209868C837D02FA5C005B
:108330005D00476C6F62616C20205461626C652047
:108340002037005283128309868C838802FA5C00EE
:108350005D00476C6F62616C20205461626C652027
:108360002038007283328309868C839302FA5C0082
:108370005D00455849542020202020202020202026
:10838000202000328252830300CD0000504F532042
:1083900030202020202020202020202000A683AA7A
:1083A000840100D00000504F532031202020202095
:1083B00020202020202000C0838C830100D10000D9
:1083C000504F532032202020202020202020202009
:1083D00000DA83A6830100D20000504F53203320DF
:1083E0002020202020202020202000F483C0830192
:1083F00000D30000504F5320342020202020202084
:1084000020202020000E84DA830100D40000504F89
:10841000532035202020202020202020202000282C
:1084200084F4830100D50000504F532036202020D3
:1084300020202020202020200042840E840100D60D
:108440000000504F532037202020202020202020C3
:108450002020005C8428840100D70000504F532066
:108460003820202020202020202020200076844238
:10847000840100D80000504F5320392020202020B4
:108480002020202020200090845C840100D900005E
:10849000504F532031302020202020202020202029
:1084A00000AA8476840100DA00004558495420204F
:1084B00020202020202020202020008C8390840356
:1084C00000CD000020545820566F6C7420204D655C
:1084D0007465722000E084628607884E5D866700BE
:1084E000545820416C61726D20566F6C74616765E1
:1084F000000085C48408C8B90286670000FF000038
:10850000526573657420426174742054696D65729C
:10851000001E85E084038CDB000867865D00205226
:108520005820566F6C7420204D6574657220003A97
:1085300085008507886A5D866700536572766F20BF
:10854000204D696E2050756C7365005A851E85023A
:10855000C8AE029867E803881300536572766F20EF
:10856000204D61782050756C7365007A853A8502DC
:10857000C8B0029867E8038813004E756D62657293
:1085800020204368616E6E656C73009E855A850578
:10859000CEA202AA6704000900325D3A5D002020E5
:1085A0002053796E6320776964746820202000BEB0
:1085B000857A8502C8A3029867C800DC05002020E0
:1085C000536869667420496E76657274202000DAFB
:1085D000859E850388CD03BC67002020466F726DA1
:1085E000617420466C617368202000F485BE8507A5
:1085F00080945D0020202020436F6E66696775724D
:1086000065202020000E86DA850980DC8600202087
:108610004A6F79537469636B2043616C2020002892
:1086200086F485098098890020202020202020467B
:108630004D532020202020200046860E86038CE902
:1086400000F666425D00204672657175656E63795D
:108650002042616E6420006286288600807C86D17C
:10866000020045584954202020202020202020208E
:10867000202000C48446860300CD00002020202056
:10868000204E6F202052462020202020009486C4B7
:10869000860000002020202020353020204D487A00
:1086A0002020202000AC867C860100002020202095
:1086B00020353320204D487A2020202000C4869485
:1086C000860200002020202020373220204D487ACA
:1086D00020202020007C86AC860300004F7574703B
:1086E0007574206368616E6E656C203100F8862CAD
:1086F00088000146880004004F757470757420630B
:1087000068616E6E656C2032001487DC860001465D
:10871000880104004F7574707574206368616E6E13
:10872000656C2033003087F886000146880204001B
:108730004F7574707574206368616E6E656C20345B
:10874000004C871487000146880304004F7574703D
:108750007574206368616E6E656C203500688730C3
:1087600087000146880404004F7574707574206397
:1087700068616E6E656C20360084874C8700014608
:10878000880504004F7574707574206368616E6E9F
:10879000656C203700A087688700014688060400C2
:1087A0004F7574707574206368616E6E656C2038E7
:1087B00000BC8784870001468807040053656C6508
:1087C00063742041696C20205472696D00D887A0C1
:1087D0008700011689B2020053656C6563742045F9
:1087E0006C6520205472696D00F487BC8700011607
:1087F00089B3020053656C65637420527564202050
:108800005472696D001088D88700011689B402007F
:1088100053656C6563742054687420205472696DCC
:10882000002C88F48700011689B502004558495488
:1088300020202020202020202020202000DC861046
:10884000880300CD00002020202041696C65726FF4
:108850006E2020202020006088FC880100DC0000C1
:1088600020202020456C657661746F7220202020C6
:10887000007A8846880200DC000020202020205258
:10888000756464657220202020200094886088032D
:1088900000DC0000202020205468726F74746C6526
:1088A0002020202000AE887A880400DC00002020F0
:1088B000202020202043483520202020202000C8D0
:1088C0008894880500DC0000202020202020204300
:1088D000483620202020202000E288AE880600DCD8
:1088E0000000202020202020204348372020202066
:1088F000202000FC88C8880700DC00002020202001
:10890000202020434838202020202020004688E2D4
:10891000880800DC0000202020204E6F20205472A8
:10892000696D202020200030897E890000DC000055
:1089300020202020205472696D203120202020200A
:10894000004A8916890100DC0000202020202054E4
:1089500072696D2032202020202000648930890235
:1089600000DC000020202020205472696D2033207C
:1089700020202020007E894A890300DC000020207E
:108980002020205472696D203420202020200016E1
:108990008964890400DC00002020202041696C6586
:1089A000726F6E202020202000B489B08A07805486
:1089B0005F15040020202020456C657661746F727D
:1089C0002020202000D08998890780545F1B050053
:1089D00020202020527564646572202020202020F1
:1089E00000EC89B4890780545F21060020202020F4
:1089F0005468726F74746C652020202000088AD03F
:108A0000890780865E2707002020202020204348F9
:108A1000362020202020202000248AEC8907808610
:108A20005E3B0000202020202020434837202020CB
:108A30002020202000408A088A0780865E3F0100AF
:108A4000202041696C65726F6E207472696D202000
:108A5000005C8A248A07809A5D2B080020456C659B
:108A60007661746F7220207472696D2000788A407C
:108A70008A07809A5D2F0900202052756464657210
:108A800020207472696D202000948A5C8A07809A85
:108A90005D330A00205468726F74746C6520207412
:108AA00072696D2000B08A788A07809A5D370B0062
:108AB000457869742020202020202020202020209C
:108AC000009889948A0300CD00002020202043656F
:108AD0006E7465722020202020200000202020526B
:108AE000696768742F446F776E2020200000202073
:108AF00020204C6566742F55702020202020000017
:108B000001000F00D20000000300D20000001E0090
:108B1000D2000080120902C802AC0194018A02D07E
:108B200001C4017A02F501C10105002502E1012815
:108B300002DE015E02B5012402E401360173005F2A
:108B4000016F000000080001040910192431405190
:108B50006400132433404B545B60636400010203E0
:108B6000060C1522334964001B31424F585E616286
:108B70006364000A141E28323C46505A64001428CC
:108B80003C5064503C28140000050A0F1419283783
:108B9000465564000F1E2D3C4B50555A5F64010A28
:108BA0000000109001FF00A5E7C009F30000DC05FC
:108BB0009411010203040000005801000102830423
:108BC00005060708090A0B0C0D0E0F000000000037
:108BD0000000000000000000000000000000000095
:108BE0000000000000000000000000000000000085
:108BF0000000000000000000000000000000000075
:108C00004D4F44454C203031202020202020202072
:108C1000000001B80B00013C190000000001B80B76
:108C200000013C190000000001B80B00013C1900D4
:108C3000000000FEA00F1901D00700FEA00F00FEEB
:108C4000A00F00FEA00F0001B80B000132FF3200A0
:108C500032003200CEFFCE00CE00CE000000001465
:108C6000140000000A0A0000000A0A0000000A0AB4
:108C70000000F4010A0000000A0A0000000A0A00CD
:108C800000000A0A0000000A0A0000000A0A0000A8
:108C9000000A0A0000000A0A000000000000000AA2
:108CA00000000000000200000000000000FF0001C2
:108CB000028304050607898B4B8C0D8E8F010008FB
:108CC0001000074B8C0400200000000000FF0D0086
:108CD00020002000200020002000000104091019BD
:108CE000243140516400132433404B545B6063646F
:108CF0000000000000000000000000000000000074
:108D0000020103040506070800000000000000003F
:108D10000000000000000000000000000000000053
:108D20000000000000000000000000000000000043
:108D30000000000000000000000000000000000033
:108D40000000000000000000000000000000000023
:108D50000000000000000000000000000000000013
:108D60000000000000000000000000000000000003
:108D700000000000000000000000000000000000F3
:108D800000000000000000000000000000000000E3
:108D900000000000000000000000000000000000D3
:108DA00000000000000000000000000000000000C3
:108DB00000000000000000000000000000000000B3
:108DC00000000000000000000000000000000000A3
:108DD0000000000000000000000000000000000093
:108DE0000000000000000000000000000000000083
:108DF0000000000000000000000000000000000073
:00000001FF
